:100000000C941E060C94F0280C941D290C944606A2
:100010000C9446060C9446060C9446060C94460630
:100020000C9446060C9446060C9422130C94460637
:100030000C9446060C9446060C9446060C94460610
:100040000C944A290C9446060C94382D0C947B2D64
:100050000C9446060C9446060C9446060C944606F0
:100060000C9446060C9446062B198D196C196F19C1
:100070007219751978197B197E198D198719BF1A8C
:10008000C11AC11ABF1AC11AC11AC11AC11AC11A9A
:10009000C11AC11AC11AC11AC11AC11AC11AC11A88
:1000A000451AC11AC11AC11AC11AC11AB619C11A00
:1000B000C11AC11AC11AC11AC11AC11AC11AC11A68
:1000C000C11AC11AC11AC11AC11AC11A511A511A38
:1000D000511A511A511A511A511A511A511AC11A58
:1000E000C11AC11AC11AC11AC11AB619501A501A26
:1000F000501A501AC11A5E1A641A6A1A701A761ABD
:100100007C1A821A881A921A9C1AA61AB01AF7191F
:10011000B919C11AC11AC11AC11A451AC11AC11A8C
:10012000C11AC11AC11AC11AC11AC11A4F1A4F1ADB
:100130004F1A4F1AC11A5E1A641A6A1A701A761A7E
:100140007C1A821A881A921A9C1AA61AB01AF719DF
:10015000B919C11AC11AC11AC11A451AF41AF41AE6
:10016000F41AF41AF41AF41AF41AF41AF41AF41A1F
:10017000F41AF41AF41A0B1C0B1C0B1C0B1C0B1C92
:100180000B1C391B431B4D1B571BB51BBF1BCE1B29
:10019000DF1B671D7C1D881D911DA01DC51DCE1D6B
:1001A000171EE01D2C21322138213F214D216F21C6
:1001B0008D21456E746572206D656E752E2E2E0034
:1001C000546F67676C6564206D6963726F50504D42
:1001D00000546F67676C656420696E76657274653C
:1001E000642050504D2100546F67676C6564205443
:1001F00058206D7574696E672100546F67676C6570
:10020000642074656C656D65747279210050726F3D
:10021000746F636F6C206572726F72207769746897
:100220002052580054696D656F7574207768656E4B
:1002300020636F6E6E656374696E6720746F205201
:100240005800507265737320616E79206B65792058
:10025000746F2063616E63656C00436F6E6E6563DF
:1002600074696E6720746F2052582C20706F776508
:100270007220757020746865205258202877697440
:10028000682062696E6420706C7567206966206EF4
:100290006F74207573696E6720616C776179732064
:1002A00062696E642900546F67676C656420276912
:1002B0006D6D656469617465206F75747075742700
:1002C00000546F67676C65642027736C61766520E6
:1002D0006D6F64652700546F67676C6564202761E4
:1002E0006C776179732062696E642700546F676769
:1002F0006C65642050504D206368616E6E656C20A3
:100300006C696D69740053657420525353492069B8
:100310006E6A656374696F6E206368616E6E656C8A
:100320002028303D3D64697361626C652900536526
:10033000742050504D206D696E696D756D20737914
:100340006E630053657420626561636F6E20696E31
:1003500074657276616C0053657420626561636FC9
:100360006E2064656C617900536574206265616319
:100370006F6E206672657175656E637920696E2097
:10038000487A3A20303D64697361626C652C205074
:10039000783D504D52206368616E6E656C20782CFC
:1003A0002046783D465253206368616E6E656C202E
:1003B00078005365742050574D2073746F7020641B
:1003C000656C61792028302064697361626C6564B2
:1003D0002C20312D323535203D3D20302E317320FB
:1003E0002D2035306D696E29005365742050504DB5
:1003F0002073746F702064656C61792028302064EC
:10040000697361626C65642C20312D323535203D75
:100410003D20302E3173202D2035306D696E29003E
:10042000536574206661696C736166652064656CF0
:1004300061792028302064697361626C65642C20C6
:10044000312D323535203D3D20302E3173202D2089
:1004500035306D696E29002A2A2A2A2A2A2A2A2A50
:100460002A2A2A2A2A2A2A2A2A2A2A2A2A2A2A2AEC
:100470002A2A2A2A0052582041636B6564202D20C5
:1004800072657665727420737563636573736675E0
:100490006C21002A2A2A2A2A2A2A2A2A2A2A2A2AAD
:1004A0002A2A2A2A2A2A2A2A2A2A2A2A2A2A2A2AAC
:1004B000002A2A2A2A2A2A2A2A2A2A2A2A2A2A2AC6
:1004C0002A2A2A2A2A2A2A2A2A2A2A2A2A2A00528E
:1004D000582041636B6564202D20757064617465DC
:1004E000207375636365737366756C21002A2A2A0D
:1004F0002A2A2A2A2A2A2A2A2A2A2A2A2A2A2A2A5C
:100500002A2A2A2A2A2A2A2A2A2A0056616C696457
:100510002063686F69636573206172653A205B319F
:100520005D2D5B31365D20286368616E6E656C20E1
:10053000312D31362900536574206F7574707574D0
:1005400020666F7220706F727420005B585D2061AE
:10055000626F7274206368616E67657320616E6498
:10056000206578697420525820636F6E6669670051
:100570005B535D20736176652073657474696E6783
:100580007320746F205258005B525D20726576654F
:1005900072742052582073657474696E6773207486
:1005A0006F2064656661756C747300557365206EA9
:1005B000756D62657273205B312D445D20746F2010
:1005C0006564697420706F727473205B452D515D92
:1005D00020666F722073657474696E677300202DD6
:1005E00020726563656976657220636F6E66696700
:1005F000757261746F722C20727820737720000AF4
:100600000A6F70656E4C52536E67200053657420FC
:1006100073657269616C2062617564726174653AB8
:10062000200056616C69642063686F696365733A82
:100630002031202D20342B34202F2032202D203823
:10064000202F2033202D20382B34202F2034202D14
:10065000203132202F2035202D2031322B34202FF5
:100660002036202D20313600536574204368616E9A
:100670006E656C20636F6E6669673A20005365741F
:100680002044617461726174652028302D32293AEA
:10069000200053657420486F70206368616E6E653A
:1006A0006C7320286D61782032342C207365706162
:1006B000726174656420627920636F6D6D61732966
:1006C0002076616C69642076616C75657320312DCC
:1006D0003235353A2000536574206368616E6E656B
:1006E0006C2073706163696E6720287831306B48C5
:1006F0007A293A200053657420524620706F77653E
:10070000722028302D37293A200053657420524634
:10071000206D6167696320286865782920652E67E8
:100720002E20307844454144463030443A2000532E
:1007300065742062617365206672657175656E63AC
:10074000792028696E20487A293A20005B5A5D207A
:10075000656E746572207265636569766572206383
:100760006F6E66696775726174696F6E2075746902
:100770006C79005B465D20646973706C61792061FF
:10078000637475616C206672657175656E63696509
:10079000732075736564005B525D2063616C6375E3
:1007A0006C6174652072616E646F6D206B65792079
:1007B000616E6420686F70206C697374005B495DC2
:1007C000207265696E697469616C697A6520736508
:1007D0007474696E677320746F20736B65746368DB
:1007E0002064656661756C7473005B585D2072658A
:1007F00076657274206368616E67657320616E64EC
:100800002065786974206D656E75005B535D20739B
:100810006176652073657474696E677320746F20E8
:10082000454550524F4D20616E64206578697420B3
:100830006D656E7500557365206E756D62657273BA
:10084000205B302D395D20746F20656469742070E1
:100850006172616D657465727300202D2053797328
:1008600074656D20636F6E66696775726174696F18
:100870006E000A0A6F70656E4C52536E672000510D
:1008800029204F7574707574206265666F726520DB
:100890006C696E6B20283D465329203A2000502970
:1008A00020536C617665206D6F64652028657870D3
:1008B0006572696D656E74616C293A20004F29205C
:1008C00054696D65642042494E44206174207374FC
:1008D000617274757020203A20004E292050504DCE
:1008E000206F7574707574206C696D69746564200F
:1008F000202020203A200044495341424C454400E6
:100900004D292050504D205253534920746F20637D
:1009100068616E6E656C202020203A20004C2920F2
:1009200050504D206D696E696D756D2073796E63E1
:10093000202875732920203A200044495341424C15
:100940004544004B29204661696C736166652062ED
:100950006561636F6E20696E74762E2028312D32AA
:10096000353573293A20004A29204661696C736144
:10097000666520626561636F6E2064656C617920D5
:1009800028302D323535203D3E20313073202D204A
:100990003135306D696E293A200049292046616958
:1009A0006C7361666520626561636F6E206672714B
:1009B0002E203A200048292050574D2073746F7024
:1009C0002064656C6179202020202020203A2000BE
:1009D00047292050504D2073746F702064656C61FE
:1009E00079202020202020203A200046292046611E
:1009F000696C736166652064656C617920202020D4
:100A00002020203A200050574D206368616E6E65AB
:100A10006C200066756E6374696F6E3A2000292041
:100A2000706F72742000506F776572546F776572C3
:100A300000445446205548462033322D62697420C4
:100A400031306368004F70656E4C52536E67525878
:100A5000206D696E6920342F36636800466C7974A6
:100A6000726F6E2F4F72616E6765525820554846FF
:100A70002038636800525820747970653A20004429
:100A8000697361626C656400487A00203D3D200016
:100A900043616C63756C61746564207061636B6540
:100AA0007420696E74657276616C3A200042292068
:100AB0004D6963726F202868616C66292050504D23
:100AC000202020203A00412920496E766572746505
:100AD000642050504D20696E20202020203A0030A4
:100AE00029204D7574652062757A7A657220286DAB
:100AF0006F73746C79293A003929205365726961E2
:100B00006C2062617564726174653A00736D617224
:100B100074506F7274004672536B79005472616E38
:100B200073706172656E740044697361626C6564B0
:100B30000038292054656C656D657472793A2020FF
:100B40002020202020003729204368616E6E656CCC
:100B500020636F6E6669673A202000362920446161
:100B60007461726174652028302D32293A2020206A
:100B700000352920486F70206368616E6E656C7364
:100B80003A2020202020003429204368616E6E65C1
:100B90006C2073706163696E673A202000332920EE
:100BA000524620706F7765722028302D37293A2001
:100BB0002020003229205246206D616769633A2067
:100BC0002020202020202020003129204261736530
:100BD000206672657175656E63793A202020000089
:100BE00000000700020100000304060000000000EE
:100BF00000000001020408102040800102040810D7
:100C00002001020408102004040404040404040263
:100C10000202020202030303030303000000002395
:100C2000002600290000000000250028002B0000FD
:100C3000000000240027002A0000EF2E11241FBE10
:100C4000CFEFD8E0DEBFCDBF13E0A0E0B1E0ECEE27
:100C5000F3E602C005900D92A83CB107D9F716E063
:100C6000A8ECB3E001C01D92A239B107E1F71CE086
:100C7000CCE3DCE004C02297FE010E94F82FCA33C7
:100C8000D107C9F70E942B2F0C94F4310C9400006B
:100C900080917705813019F482E080937705809107
:100CA0007705833019F484E0809377050895A8953B
:100CB0000895DC01ED91FC910190F081E02D099502
:100CC00008952091780530917905382748E0C901C9
:100CD000880F991F37FF06C09C0151E2252750E17C
:100CE000352701C09C01415091F73093790520933D
:100CF0007805089588E380937A0580E092ECA1E07E
:100D0000B0E080937B0590937C05A0937D05B09324
:100D10007E0587E08093870580EC9AECA9E8B6E32E
:100D200080937F0590938005A0938105B093820501
:100D300085E0809388058DEE9EEFADEABEED809351
:100D4000830590938405A0938505B0938605E9E813
:100D5000F5E080E090E0863028F4DC01AE54BC4F32
:100D60002C9101C020E0219301968831910599F7DB
:100D700082E08093A1058AE08093A205089580EC2B
:100D800097EFAAEBB7E38093BF059093C005A093BC
:100D9000C105B093C20580E090E0A0E0B0E580938B
:100DA000C3059093C405A093C505B093C605E7ECB1
:100DB000F5E080E081938F5F8031E1F70895A0E056
:100DC000B0E0E5EEF6E00C94C12FD82F0E94A029E8
:100DD0006115710581059105C9F30E946430109277
:100DE0008305109284051092850510928605C4E053
:100DF000812C912C54018A94C0908305D090840555
:100E0000E0908505F0908605FE2CED2CDC2CCC24A2
:100E10000E945F30A50194010E94A02F6C0D7D1DE2
:100E20008E1D9F1D609383057093840580938505B7
:100E300090938605C15001F7DD2309F450C009E8FD
:100E400015E0E801A12CB12C62E3C62ED12CE12CD7
:100E5000F12C8881882309F442C0B39419F40E94CC
:100E60007A063DC00E945F30A70196010E94A02F24
:100E7000E1E0E60FA9E8B5E08A2F801B8A1520F48F
:100E80008D918E13F9CFE9CF2091880530E0A0E154
:100E9000B7E20E94382F9B01AC01AE2FB0E00E9458
:100EA000472F40907F05509080056090810570909D
:100EB0008205640D751D861D971D4090BF055090DD
:100EC000C0056090C1057090C205461657066806B9
:100ED000790618F2E993A39488E1A812BACFCDB7A6
:100EE000DEB7E0E10C94DD2F8436910520F4BC01DF
:100EF00080E090E017C09C018E3B910528F42A55B4
:100F00003109AAE0B0E00CC0823D910528F4245BD1
:100F10003109A4E6B0E004C02D5C3109A8E5B2E0D7
:100F20000E94382FA4E6B0E09B01AC010E94472F3D
:100F3000089590E08C599F4F0E947407089561E0D6
:100F400086E00E944D2A60E086E00E94862A82E0C8
:100F50008093B00085E08093B10061E083E00E945F
:100F60004D2A60E083E00E94862A0895CF93DF93A4
:100F7000EC010097E9F061E086E00E94862A9E017C
:100F800040E050E068E478EE81E090E00E94A02F1D
:100F90002F3F31054105510529F020F02FEF30E0BA
:100FA00040E050E02093B3008091B000806107C022
:100FB00060E086E00E94862A8091B0008F7E809358
:100FC000B000DF91CF91089560E08EE00E944D2A3D
:100FD00061E08FE00E944D2A61E080E10E944D2A8D
:100FE00060E082E00E944D2A61E084E00E944D2A88
:100FF000089542E050E068E476E080E00E94D02866
:101000000895E3E0F0E089E080935700E491E67012
:1010100081E0E63009F080E00895CF93DF93C82F98
:101020000E940108882381F0DFB781E08093760574
:10103000F8940E94570688E180936000C093600096
:10104000C1110E945706DFBFDF91CF9108958F92A3
:101050009F92AF92BF92CF92DF92EF92FF92CF9387
:10106000FC01C0A5EC2FE770F0E0E658FC4FA08132
:10107000B0E0C7FF03C024E130E002C02FE030E061
:10108000FC0197A183E1989FF0011124E25CFE4FDF
:1010900080809180A280B380A20FB31F20E43FE143
:1010A0004DE750E00E94522FA50194010E947E2F2F
:1010B0008C2F887149F469017A01E0EDCE0EE7E0EA
:1010C000DE1EE11CF11C1BC0C7FF05C060E47AE80E
:1010D0008CE29EE004C060E07EEE8AEB9BE069015A
:1010E0007A01F8EBCF0EFBE0DF1EE11CF11CA5013D
:1010F00094010E947E2FC20ED31EE41EF51EC7016E
:10110000B60169517C4F8F4F9F4F28EE33E040E08E
:1011100050E00E947E2FA8EEB3E00E94472FCF91AF
:10112000FF90EF90DF90CF90BF90AF909F908F9007
:1011300008958F3F910551F048F0811522E0920704
:1011400038F08115934030F482E0089580E00895EE
:1011500081E0089583E00895A0E0B0E0E2EBF8E0DC
:101160000C94CA2FEB018A01B82FB695A0E0288114
:101170003981F80120832A813B8121832C813D81A3
:1011800022832E813F812383688179814A815B811B
:101190002C813D81EE81FF819F2F9295990F990FB0
:1011A000907C272F2370922B252F2370220F220F44
:1011B000922B232F23702295207F922BF80194836A
:1011C0000B5F1F4F2896AF5FBA1788F680FF24C0C9
:1011D000888199810E949908D82E8A819B810E94DA
:1011E0009908E82E8C819D810E949908F82E8E81A5
:1011F0009F810E949908F0E4DF9EA001112490E1F4
:10120000E99E90011124242B282BE4E0FE9EB001DE
:101210001124262BF8012083CDB7DEB7E7E00C942C
:10122000E62F803223E0920708F1883E23E0920700
:1012300040F48F519340E4E096958795EA95E1F765
:101240000895803D27E0920718F48C5D934008953F
:10125000883928E0920768F4885C974074E0969596
:1012600087957A95E1F78D509C4F089580E090E046
:1012700008958FEF93E008958C30910540F4A4E039
:10128000880F991FAA95E1F7885D9C4F0895843FC8
:1012900023E0920718F484529C4F0895811524E0AE
:1012A000920740F48657934FF4E0880F991FFA9500
:1012B000E1F7089580E998E008959C013695279517
:1012C00025753575821B930B9C012373337396959B
:1012D00087959695879583739373820F931F9C01CF
:1012E00054E0369527955A95E1F7280F391F2F704E
:1012F0003F7041E051E0249FC001259F900D349F35
:10130000900D1124892F08954298882319F0000028
:10131000419A02C0000041980000429A00000895DE
:10132000429A000086B14298000081700895CF93E0
:10133000DF93D82F5C9A42985C98C8E08D2F807814
:101340000E948409DD0FC150C9F74298DF91CF9107
:1013500008958F770E9497090895CF93DF93D82F30
:10136000C8E08D2F80780E948409DD0FC150C9F735
:101370004298DF91CF910895CF93DF934298C8E0D0
:1013800080E0D82FDD0F0E9490098D0FC150C9F762
:10139000DF91CF9108950E94A9090E94BC095C9A2F
:1013A0000895A1E0B0E0E7EDF9E00C94CF2F80685C
:1013B00069830E9497096981862F0E94AD095C9A12
:1013C0002196E2E00C94EB2FCF93C0918305C827C0
:1013D000E82FF0E0E658FA4F678589E70E94D109C7
:1013E0006C2F8DE30E94D1096C2F82E40E94D109F9
:1013F000CF91089586E20E94CB090895CF93DF93A1
:10140000EC016C818CE10E94D1096D818DE10E941B
:10141000D1096E818EE10E94D1096F8180E20E9424
:10142000D109688581E20E94D109698582E20E9422
:10143000D1096A8583E20E94D1096B8584E20E940A
:10144000D1096C8585E20E94D1096D858AE20E94EE
:10145000D1096E858EE60E94D1096F858FE60E94C4
:10146000D109688980E70E94D109698981E70E94D2
:10147000D1096A8982E70E94D109DF91CF9108954D
:10148000CF92DF92EF92FF92CF93DF936B017C01BB
:10149000C11488E3D8068CE9E8068CE1F80628F543
:1014A000C701B60120E836E948E950E00E947E2FE6
:1014B000E901689760E879E687E69FEF0E945A2F76
:1014C0006C0D7D1D8E1D9F1DF2E0660F771F881F1E
:1014D000991FFA95D1F721E732E040E050E00E94F1
:1014E0007E2FF22EE32E80E421C0C701B60120E05A
:1014F0003DE241E351E00E947E2FE901689760E000
:1015000073ED8EEC9EEF0E945A2F6C0D7D1D8E1D8B
:101510009F1D660F771F881F991F21E732E040E06B
:1015200050E00E947E2FF22EE32E80E66C2F6F712A
:10153000680F85E70E94D1096E2D86E70E94D109C8
:101540006F2D87E70E94D109DF91CF91FF90EF9037
:10155000DF90CF900895682F8DE60E94D1090895FD
:101560008F929F92AF92BF92CF92DF92EF92FF92B3
:10157000CF93DF93D82F83E00E94CB09809375052A
:1015800084E00E94CB098093740560E086E00E94AD
:10159000D10961E087E00E94D1096FE789E00E94EC
:1015A000D10965E08AE00E94D10962E18BE00E94E6
:1015B000D10965E18CE00E94D1096DEF8DE00E94B8
:1015C000D10960E08EE00E94D109DD2319F08BE2A1
:1015D00091E008C02091A10533E1239FC0011124AF
:1015E000825C9E4F0E94FE096CE880E30E94D10954
:1015F0006FE082E30E94D10962E483E30E94D10993
:101600008091A20587FF02C064E101C06AE084E323
:101610000E94D1096AE285E30E94D1096DE286E366
:101620000E94D10964ED87E30E94D10960E088E35C
:101630000E94D10960E089E30E94D109D11109C05B
:10164000C0908305D0908405E0908505F0908605D4
:1016500007C0C5E9CC2EC1ECDC2EED2CCEEDFC2E66
:10166000CAE38F2C9924AA24BB24682D8C2F0E94B6
:10167000D109682D85E08C0F0E94D109FE2CED2C3C
:10168000DC2CCC24CF5FCE3361F76FEF83E40E9474
:10169000D1096FEF84E40E94D1096FEF85E40E94C5
:1016A000D1096FEF86E40E94D109DD2311F066E0D5
:1016B00002C0609187058DE60E94D10960E089E74C
:1016C0000E94D109609188058AE70E94D10960E0F3
:1016D00083E70E94D10960E084E70E94D109D1111B
:1016E00009C060917F05709180058091810590917E
:1016F000820504C060EC7AEC89E896E30E94400A17
:10170000DF91CF91FF90EF90DF90CF90BF90AF909F
:101710009F908F90089561E087E00E94D10964E274
:101720008EE70E94D10963E088E00E94D10960E061
:1017300088E00E94D10965E087E00E94D10962E05B
:1017400085E00E94D10983E00E94CB098093750552
:1017500084E00E94CB0980937405089583E00E9481
:10176000CB098093750584E00E94CB0980937405B2
:1017700061E087E00E94D1096AE070E080E090E0DB
:101780000E94C3290E948B0B00000895CF92DF9224
:10179000FF920F931F93CF93DF931F92CDB7DEB7C6
:1017A000082F162F8EE399830E94D109F02EC02EA8
:1017B0009981D92E8C2D8F19811738F4F6016191FA
:1017C0006F018FE70E94D109F5CF64E085E00E94A8
:1017D000D10983E00E94CB098093750584E00E94C3
:1017E000CB09809374050E94A029609370057093C3
:1017F0007105809372059093730569E087E00E94FC
:10180000D10981E0809377050F90DF91CF911F91EF
:101810000F91FF90DF90CF9008950F931F930E9438
:10182000C60B80917705813099F40E94A029009120
:101830007005109171052091720530917305601B40
:10184000710B820B930B603A76488140910548F307
:1018500080917705813031F46EE971E086EE95E094
:101860000E948C2B1F910F9108950F931F938091CD
:101870007705823021F41092770581E020C08091B5
:1018800077058130D9F40E94A0290091700510914C
:1018900071052091720530917305601B710B820BED
:1018A000930B613A76488140910540F061E087E012
:1018B0000E94D1091092770582E001C080E01F915B
:1018C0000F910895CF93DF93EC014AE050E06D2F24
:1018D00070E086EE95E00E945A2C6EE286EE95E06E
:1018E0000E945E2BBE0184E0769567958A95E1F7AC
:1018F0006F7077274AE050E086EE95E00E945A2C00
:101900006EE286EE95E00E945E2BBE016F70772737
:101910004AE050E086EE95E00E945A2CDF91CF918C
:101920000895D82FC0E0CD1790F4439A299A64E621
:1019300070E080E090E00E94C3294398299864E613
:1019400070E080E090E00E94C329CF5FECCF6CE2B2
:1019500071E080E090E00E94C329E4CF0F931F93D1
:10196000CF93DF93EC01062F15E0115051F0CE011B
:101970000E94DB31081741F0602FCE010E94E33155
:10198000F4CF82E00E94910CDF91CF911F910F91D3
:101990000895A0E0B0E0EFECFCE00C94C12F482EDD
:1019A000562EC0E0D0E0612C712CE12CF12C00E02F
:1019B00010E041100CC06090D80586E4689E3001AC
:1019C000112459E1E52EF12C0EEB15E01EC091E03B
:1019D00049120FC06090D805E6E46E9E30011124D4
:1019E000FBE16F0E711C49E2E42EF12C0AE715E0D1
:1019F0000CC082E0481209C028E1622E772473945B
:101A0000EE24E394F12C07ED15E043018C0E9D1EAE
:101A100010927905109278053401A62CA818B12CE3
:101A2000C30101966C01AE14BF04A8F4A00EB11E50
:101A3000511006C0C3010E94DB31F501808305C04F
:101A4000F5016081C3010E94AE0CF50180810E9406
:101A500061063601E2CFC301511018C0C3010E94D4
:101A6000DB31B82EC6010E94DB312B2D30E0322F46
:101A70002227282B8091780590917905821793076A
:101A800079F4C0E0D0E05524539493CF36016091AF
:101A900079050E94AE0C60917805C6010E94AE0CDB
:101AA000C05EDE4FC13E92E0D90708F482CF852D9B
:101AB000CDB7DEB7E0E10C94DD2F61E082E00E945B
:101AC000C90C089560E082E00E94C90C8091D7059E
:101AD000853020F01092D7050E945D0D8091D705CA
:101AE0008093D805089561E080E00E94C90C61E010
:101AF00081E00E94C90C089560E080E00E94C90C5A
:101B0000882351F060E081E00E94C90C882321F015
:101B100080917A05883349F00E94BF060E947A06B8
:101B200081E00E94DF060E94730D0895882319F05A
:101B30006AEA71E002C06EEA71E086EE95E00E940A
:101B40008C2B0895FF920F931F93CF93DF9369EC33
:101B50007BE086EE95E00E94382B40917F05509106
:101B6000800560918105709182052AE030E086EE63
:101B700095E00E94612C63EB7BE086EE95E00E948D
:101B8000382B4091830550918405609185057091B3
:101B9000860520E130E086EE95E00E94612C6DE93B
:101BA0007BE086EE95E00E94382B4AE050E06091A1
:101BB000870586EE95E00E94892C67E87BE086EE3B
:101BC00095E00E94382B4AE050E06091880586EE4F
:101BD00095E00E94892C61E77BE086EE95E00E940B
:101BE000382BC9E8D5E0F12C8E0188818823A9F033
:101BF000FF2031F061EB71E086EE95E00E945B2BF7
:101C000021964AE050E0F801608186EE95E00E945E
:101C1000522CF394F8E1FF12E7CF86EE95E00E9494
:101C2000662B6BE57BE086EE95E00E94382B4AE060
:101C300050E06091A10586EE95E00E94892C66E453
:101C40007BE086EE95E00E94382BE091A205E770DC
:101C5000F0E0EE0FFF1FEE57FC4F6081718186EEC2
:101C600095E00E948C2B61E37BE086EE95E00E947C
:101C7000382B8091A2058871883069F028F4811191
:101C800013C068E27BE00CC0803141F0883161F420
:101C90006CE07BE005C06CE17BE002C066E17BE0CC
:101CA00086EE95E00E947A2B68EF7AE086EE95E06A
:101CB0000E94382B40917B0550917C0560917D05F9
:101CC00070917E052AE030E086EE95E00E94612C5E
:101CD0006FED7AE086EE95E00E94382B8091C30587
:101CE00080710E94960D66EC7AE086EE95E00E9487
:101CF000382B8091C30580740E94960D6DEA7AE0BE
:101D000086EE95E00E94382B8091C30580720E9478
:101D1000960D60E97AE086EE95E00E94382B8AE71E
:101D200095E00E942708AB01BC012AE030E086EE76
:101D300095E00E94432C6BE87AE086EE95E00E94E5
:101D4000382B8AE795E00E9427089B01AC0160E4EC
:101D500072E48FE090E00E947E2FBA01A9012AE090
:101D600030E086EE95E00E94432C68E87AE086EE4B
:101D700095E00E947A2BCDB7DEB7E5E00C94E82F12
:101D80008F929F92AF92BF92CF92DF92EF92FF928B
:101D9000811107C06FE77AE086EE95E00E947A2B0A
:101DA0002FC090E00E94740724E630E040E050E04D
:101DB0000E947E2FCA01B9012AE030E040E050E0E5
:101DC0000E947E2F49015A016B017C012AE030E01C
:101DD000B501A40186EE95E00E94432C6EE286EEEA
:101DE00095E00E945E2B2AE030E0B701A60186EE66
:101DF00095E00E94432C63E786EE95E00E949E2BBF
:101E0000FF90EF90DF90CF90BF90AF909F908F901A
:101E100008951F93CF93DF9365E77AE086EE95E010
:101E20000E94382B8091A305813041F46CE57AE063
:101E300086EE95E00E947A2B10E050C0823019F4B3
:101E400065E47AE0F5CF843019F461E37AE0F0CF0D
:101E5000853091F766E27AE0EBCFC12FD0E0C93050
:101E6000D1050CF441C068E3610F86EE95E00E9455
:101E70005E2B6EE17AE086EE95E00E94382BBE0183
:101E80006F5F7F4F4AE050E086EE95E00E94222C83
:101E900063E17AE086EE95E00E94382BCD55DA4F6B
:101EA000E981E03218F566E07AE086EE95E00E947E
:101EB000382B8981803130F06DE673E086EE95E055
:101EC0000E945B2B69816F7070E06F5F7F4F4AE00B
:101ED00050E086EE95E00E942B2C1F5F80914C0510
:101EE000181708F4BACF0FC061E3BECFEF70F0E06F
:101EF000EE0FFF1FEE56FC4F6081718186EE95E07C
:101F00000E948C2BEACF6BEE79E086EE95E00E9482
:101F1000382B8091BB050E94C00E60ED79E086EE03
:101F200095E00E94382B8091BC050E94C00E65EBA5
:101F300079E086EE95E00E94382B8091BD050E94E5
:101F4000C00E6AE979E086EE95E00E94382B409158
:101F5000B3055091B4056091B5057091B605411572
:101F600051056105710539F12AE030E086EE95E012
:101F70000E94612C67E679E086EE95E00E94382B9E
:101F80008091B7050E949907AB01BC012AE030E0BF
:101F900086EE95E00E94612C63E479E086EE95E0A0
:101FA0000E94382B4AE050E06091B80586EE95E03B
:101FB0000E94892C06C06AE379E086EE95E00E94D3
:101FC0007A2B6DE179E086EE95E00E94382B6091E6
:101FD000B9057091BA054AE050E086EE95E00E949E
:101FE000732C60E079E086EE95E00E94382B6091DA
:101FF000B205603450F470E06F5F7F4F4AE050E00C
:1020000086EE95E00E942B2C06C067EF78E086EE06
:1020100095E00E947A2B6AED78E086EE95E00E94CA
:10202000382B8091B10580FF03C063EB71E002C0E3
:1020300067EB71E086EE95E00E948C2B6DEB78E00B
:1020400086EE95E00E94382B8091B10582700E9447
:10205000960D6EE978E086EE95E00E94382B80912F
:10206000B10584700E94960D6FE778E086EE95E0EA
:102070000E94382B8091B10588700E94960DDF91E7
:10208000CF911F9108950F931F93CF93DF932091CA
:1020900049052F3FA9F56FEF75E086EE95E00E94A8
:1020A000382B88E893E00E94620C6EED75E086EEB6
:1020B00095E00E94382B80914A0590914B050E9433
:1020C000620C6BEA75E086EE95E00E947A2B68E878
:1020D00075E086EE95E00E947A2B60E775E086EE6B
:1020E00095E00E947A2B6BE475E086EE95E00E9405
:1020F0007A2B86EE95E00E94662B0E94090F68C03D
:1021000012160CF065C0332727FD309580914C05E1
:1021100090E0821793070CF45BC066E375E086EEEF
:1021200095E00E94382B60914905772767FD7095EF
:102130004AE050E086EE95E00E942B2C6BE075E0C3
:1021400086EE95E00E94382B10E008E280914D0564
:102150001817D0F5C12FD0E0CC0FDD1FC25BDA4FCE
:10216000288130E080914905992787FD9095019756
:102170002817390739F56BEB71E086EE95E00E9480
:102180005B2B4AE050E0602F86EE95E00E94522CD7
:102190006FEB71E086EE95E00E945B2BE981EF70BA
:1021A000F0E0EE0FFF1FEE56FC4F6081718186EE6E
:1021B00095E00E945B2B63EC71E086EE95E00E9457
:1021C0005B2B0F5F1F5FC2CF86EE95E00E94662BF0
:1021D000DF91CF911F910F910895FF920F931F935D
:1021E000CF93DF93C9E8D5E0F12C8E018881882355
:1021F000D1F165EC71E086EE95E00E945B2B4AE040
:1022000050E06F2D86EE95E00E94522C62ED71E059
:1022100086EE95E00E945B2B2196F801208130E04C
:10222000A0E1B7E20E94382F9B01AC01A091880584
:10223000B0E00E94472FAB01BC0180917F059091D7
:102240008005A0918105B0918205480F591F6A1F32
:102250007B1F2AE030E086EE95E00E94612CF3942B
:10226000F8E1FF12C2CFCDB7DEB7E5E00C94E82F5E
:102270001092E30485E6E4EEF4E0DF011D928A9516
:10228000E9F70895CF93C82F8F3719F0883009F0F8
:1022900045C0E091E304EE23D9F1E150E093E3047B
:1022A000F0E0EC51FB4F10826DE070E086EE95E0BF
:1022B0000E945906C0E08091E304C81760F4EC2F37
:1022C000F0E0EC51FB4F608170E086EE95E00E94FB
:1022D0005906CF5FF0CF60E270E086EE95E00E9495
:1022E00059066DE070E086EE95E00E945906C0E068
:1022F0008091E304C81778F5EC2FF0E0EC51FB4F28
:10230000608170E086EE95E00E945906CF5FF0CFC5
:1023100067E086EE95E00E945E2B1DC08B3119F4BC
:102320000E9438111AC08D30C1F08A30B1F080910E
:10233000E304843668F76C2F70E086EE95E00E9427
:102340005906E091E30481E08E0F8093E304F0E00E
:10235000EC51FB4FC08380E001C081E0CF91089534
:10236000CF93C82F0E94A0296093CC047093CD0412
:102370008093CE049093CF04C093E104CC2329F042
:1023800040E051EE60E070E004C040E855E260E0FB
:1023900070E086EE95E00E94E82DCF91089590912F
:1023A000D004492F4F7050E0BA016F5F7F4F292F43
:1023B00030E0E4E035952795EA95E1F76217730779
:1023C00059F0FA01EF52FB4F808381E0890F8F7043
:1023D000907F892B8093D00408956EE770E086EE9D
:1023E00095E00E9459060895A3E1B1E0EAEFF1E11A
:1023F0000C94C22FE9E8F5E0712C8191882321F03B
:10240000739428E17212F9CF66ED71E086EE95E0E3
:102410000E948C2B4AE050E0672D86EE95E00E94EA
:10242000892C80E00E94B00A0E948B0B8E010E5F07
:102430001F4FC12CD12C7601C39466246A945C2C66
:102440000E9494294B015C012091880530E0A0E1B5
:10245000B7E20E94382F9B01AC01C701B6010E9470
:102460005A2F20917F053091800540918105509130
:102470008205620F731F841F951F2091BF05309145
:10248000C0054091C1055091C2052617370748077E
:10249000590718F4F80160822AC08C2D0E94E409C3
:1024A00061E070E080E090E00E94C329F8011082B2
:1024B0000E949429681979098A099B09643F71402F
:1024C0008105910540F40E94FA09F801908198175E
:1024D00078F78083EDCF85B150FE05C08B7D85B93F
:1024E000439A299A04C0846285B9439829982FEFAA
:1024F000C21AD20AE20AF20A0F5F1F4F8FEFC81604
:10250000D104E104F10409F09ACFCE019395FC01C6
:10251000D82E7FEF68EC2E2F281B271510F051E0E6
:1025200056C0DE01129651E02FEF41E03D91321787
:1025300010F0322F01C0452F5F5F5F3F11F0232F56
:10254000F5CF4193242F30E0A1E0B0E0AC0FBD1FE8
:10255000A20FB31F5C93413079F0DE01A20FB31FCD
:102560005C93423049F0AFEFBFEFAC0FBD1FA20F3D
:10257000B31F6C934E3F78F6A2E0B0E0AC0FBD1FE6
:10258000A20FB31F7C934D3F30F6A3E0B0E0AC0F39
:10259000BD1FA20FB31F6C93BECF452F242F30E079
:1025A000FC01E20FF31F6081AFEFB0E0AC0FBD1F85
:1025B000A20FB31F2C91621748F44150DC01A40F05
:1025C000B11D2C9120836C934111E8CF5F5F5715AB
:1025D00020F3372D369520E0231770F4DC01A20F8D
:1025E000B11D4C91522F530FFC01E50FF11D50818D
:1025F0005C9340832E5FF0CFF9E8EF2EF5E0FF2EDD
:102600008C01802F8D19871598F4F801C1908F01E6
:102610004AE050E06C2D86EE95E00E94522C6CE270
:1026200086EE95E00E945E2BF701C1927F01E9CF13
:1026300086EE95E00E94662B81E0CD5EDE4FEFE0F6
:102640000C94DE2F1F920F920FB60F9211241F933E
:102650002F933F934F935F936F937F938F939F93AA
:10266000AF93BF93CF93DF93EF93FF93C091860017
:10267000D091870080918704909188042091A904CB
:10268000211155C09E01281B390B8091C3059091E3
:10269000C405A091C505B091C60585FD02C036955B
:1026A0002795253C49E03407B8F140910A0150E0F4
:1026B00060E070E02CE1B695A795979587952A95EF
:1026C000D1F70097A105B10521F481E090E0A0E0E9
:1026D000B0E084179507A607B707D8F480910A01E0
:1026E0008F3FB9F040E080910A01481780F4842FB1
:1026F00090E0880F991FFC01E757FB4F2081318143
:10270000FC01E55FFE4F318320834F5FECCF1092D9
:10271000AA0410920A010BC02D3B82E0380720F07A
:1027200080910A018031D8F08FEF80930A01D09315
:102730008804C0938704FF91EF91DF91CF91BF91FF
:10274000AF919F918F917F916F915F914F913F9149
:102750002F911F910F900FBE0F901F901895109101
:102760000A0181E0810F80930A01C9010E941109C9
:10277000E12FF0E0EE0FFF1FE757FB4F91838083BF
:10278000D6CF83E0809380008AE980938100809196
:10279000C30586FD05C0809181008064809381001F
:1027A0008FEF9FEF909389008093880080916F0056
:1027B000806280936F000895CF93DF930E94620D33
:1027C0008091D805843039F58BE00E94B92AC1E0A8
:1027D000D0E0892B11F4C0E0D0E08CE00E94B92A4F
:1027E000892B19F082E090E002C080E090E08C2B11
:1027F0009D2B8230910539F08330910539F0019796
:1028000039F481E006C01092D80505C082E001C00D
:1028100083E08093D805DF91CF9108956F3018F051
:1028200086958058089589E0689F802D1124089529
:10283000A0E0B0E0EEE1F4E10C94C92FC82F0E94B3
:10284000A029009138041091390420913A04309164
:102850003B046B017C01C01AD10AE20AF30A97011A
:10286000860149E8C41643E1D406E104F10410F0FE
:1028700010923C04609338047093390480933A04B6
:1028800090933B042091A9048FEF820F8230E8F5EA
:10289000E0913C04EE2309F46EC1E13011F482E0D2
:1028A000D8C1E03178F581E08E0F80933C04F0E0F0
:1028B000E757FB4FC083803109F0D4C1EBE8F4E067
:1028C000213029F4A181A695A695808108C0808138
:1028D0009181A92FA695A695A69596958795A03145
:1028E00048F4B0E090E0AA0FBB1FA55FBE4F119661
:1028F0009C938E931092AA04329684E0E939F807EB
:10290000F9F6B0C110923C04ADC1233009F023C1E7
:10291000E0913C04E11118C0CF3009F011C10E94D0
:1029200094290091B7041091B8042091B904309112
:10293000BA04601B710B820B930B62307105810529
:10294000910508F089C1FCC0E83148F481E08E0FA0
:1029500080933C04F0E0E857FB4FC083F1C0E831BE
:1029600009F0ECC0C111EAC040E050E0ABE0CA01A0
:10297000B3E0880F991FBA95E1F7A49F9001A59F36
:10298000300D1124F901E757FB4F6081E1817E2F63
:10299000777075956795FC01EE0FFF1FE55FFE4FA1
:1029A00071836083F901E657FB4FB081B695B69508
:1029B000B695E181FE2FF295FF0FF07E6F2F6B2B06
:1029C000E695E695E6957E2F777075956795FC01FF
:1029D000EE0FFF1FE35FFE4F71836083F901E55740
:1029E000FB4FB081B295B695B695B370C181DC2F1F
:1029F000DD0FDD0F6D2F6B2BC295C695C695C3708D
:102A0000E281E170EE0FEE0F7E2F7C2B75956795BE
:102A1000FC01EE0FFF1FE15FFE4F71836083F90140
:102A2000E357FB4FB081B695E181FE2FF795FF2765
:102A3000F7956F2F6B2BE6957E2F777075956795C1
:102A4000FC01EE0FFF1FEF5EFE4F71836083F90103
:102A5000E257FB4FB081B295BF70E181FE2FF29536
:102A6000F07F6F2F6B2BE295EF707E2F777075954F
:102A70006795FC01EE0FFF1FED5EFE4F71836083D3
:102A8000F901E157FB4FB081BB1FBB27BB1FC181C1
:102A9000DC2FDD0F6D2F6B2BCC1FCC27CC1FE281E1
:102AA000E370EE0F7E2F7C2B75956795FC01EE0F82
:102AB000FF1FEB5EFE4F71836083F901EF56FB4F02
:102AC000B081B695B695E181FE2FF295FF0FFF0F0D
:102AD000F07C6F2F6B2BE695E6957E2F77707595C2
:102AE0006795FC01EE0FFF1FE95EFE4F7183608367
:102AF000F901EE56FB4F20812295269527703181F2
:102B0000E32FEE0FEE0FEE0F6E2F622B732F7295E9
:102B10007695777075956795FC01EE0FFF1FE75E60
:102B2000FE4F718360834F5F5F4F4230510509F064
:102B30001ECF80919F0483FF1092AA0410923C0440
:102B40000E9494296093B7047093B8048093B904E9
:102B50009093BA0487C0243009F084C060913C048B
:102B600061110BC0C83AB1F4109279051092780542
:102B700088EA0E94610681E06CC0613019F4C0935C
:102B8000370404C0623031F4C09336048C2F0E94A5
:102B900061065AC0E09136042E2F30E0220F331F19
:102BA000462F50E0C9010296841795073CF0633226
:102BB00068F7FA01EA57FB4FC083E8CF2D5F3F4F1C
:102BC0008C2F90E06091780570917905421753073A
:102BD00049F4982F88278627972790937905809323
:102BE000780532C06817790769F58091370481301C
:102BF00049F5E13118F080E180933604F090360415
:102C0000CAE8D4E000E010E00F15D0F4FE013197DF
:102C1000808190E0982F88272881822B63E0969509
:102C200087956A95E1F70E941109F801EE0FFF1FE1
:102C3000E55FFE4F918380830F5F1F4F2296E4CFA5
:102C40001092AA0410923C0480913C04882351F015
:102C50008F5F80933C0406C080913C048F5F80931B
:102C60003C046ECFCDB7DEB7E8E00C94E52FCF93F0
:102C7000DF93E82FF0E0E254FA4FE185E03150F4C1
:102C8000F894F0E0EE0FFF1FE55FFE4F8081918129
:102C900078945DC08EE08E0F8B3058F4F0E0E25FE8
:102CA000F10924E62E9FC0012F9F900D11240C9650
:102CB0004EC0E03F09F446C038F4E13181F0E23122
:102CC00091F0E03139F409C0ED3FB1F1EE3FB9F1D7
:102CD000E13F79F180E092E03AC082E101C083E116
:102CE0000E94E22A34C08BE00E94B92AC1E0D0E001
:102CF000892B11F4C0E0D0E08CE00E94B92A892B26
:102D000019F082E090E002C080E090E08C2B9D2BD7
:102D10008230910541F08330910541F00197A9F08F
:102D200086EA92E014C08CE090E011C089E591E061
:102D30000EC086E090E00BC08AEF93E008C08FEFF2
:102D400093E005C080E090E002C084EF93E0DF9163
:102D5000CF910895A2E2B0E0E0EBF6E10C94BF2F32
:102D60009E012F5F3F4F80E1D9011D928A95E9F7BF
:102D700064E072E086EE95E029A33AA30E948C2BD2
:102D80000E94AE0B1D8A1E8A1F8A188E312C212CA0
:102D900000E0812C912C540170EC472E7DE9572ED8
:102DA00078E5672E75E3772EE0E5CE2EE3ECDE2E98
:102DB000E12CF12C84EF91E0A0E0B0E08D8F9E8FAC
:102DC000AF8FB8A380EC97EFAAEBB7E3898F9A8F08
:102DD000AB8FBC8F80EC9DE9A8E5B5E3898B9A8B1E
:102DE000AB8BBC8B86EE95E00E94A02C892B09F45E
:102DF000E1C086EE95E00E94CD2C9C0133272C3259
:102E0000310509F442C0ACF42332310509F0ABC0FE
:102E100019821A821B821C821D821E821F821886C2
:102E200019861A861B861C861D861E861F86188A92
:102E300060C02434310529F02335310509F4B2C0CE
:102E400092C064E486EE95E00E945E2B2AE030E0BA
:102E500040EC5DE968E575E386EE95E00E94EC2BB9
:102E60006CE286EE95E00E945E2B2AE030E040ECBA
:102E700057EF6AEB77E386EE95E00E94EC2B6CE26D
:102E800086EE95E00E949E2BADCF0F5F043009F0D7
:102E9000A9CF29813A814B815C81A8EEB3E00E94E1
:102EA000472F698B7A8B8B8B9C8B2D813E814F8139
:102EB00058850E94472F698F7A8F8B8F9C8F298529
:102EC0003A854B855C852D8F3E8F4F8F58A32D857E
:102ED0003E854F8558890E94472F6B017C016032E7
:102EE0003EE473078105910530F462E38CE10E94B2
:102EF000D10900E077CF603345E77407810591057C
:102F000010F462E2F3CF60345CE975078105910546
:102F100010F466E2EBCF80E5C81683ECD806E10436
:102F2000F10410F462E1E2CF90E6C9169AEED906F8
:102F3000E104F10410F465E1D9CFA0E7CA16A1E1DC
:102F4000DA06A1E0EA06F10410F461E0CFCFB0EABE
:102F5000CB16B6E8DB06B1E0EB06F10410F463E053
:102F6000C5CF65E0C3CF10ED180F1A3008F03ACF87
:102F7000E1E0F0E0EC0FFD1F24E0029FE00DF11D09
:102F800011242081318142815381AAE0B0E00E9466
:102F9000472F610F711D811D911D60837183828395
:102FA000938320CF49885A886B887C88812C912C08
:102FB000540118CF81149104A104B10489F4C30110
:102FC000B2010E94400A61E070E080E090E00E945F
:102FD000C3291D8A1E8A1F8A188E312C22242A9406
:102FE0008D8D9E8DAF8DB8A188169906AA06BB0659
:102FF000D0F40E94FA092D893E894F89588D280FF7
:10300000311D411D511D2D8B3E8B4F8B588F381616
:1030100008F4382E821508F4282E3FEF831A930AFD
:10302000A30AB30A56C0C301B20128EE33E040E060
:1030300050E00E947E2FBA01A9012AE030E086EE1E
:1030400095E00E94432C6CE286EE95E00E945E2B98
:103050004AE050E0632D86EE95E00E94522C6CE22F
:1030600086EE95E00E945E2B6D897E898F89988D12
:10307000A50194010E947E2FBA01A9012AE030E047
:1030800086EE95E00E94432C6CE286EE95E00E946D
:103090005E2B4AE050E0622D86EE95E00E94522CB5
:1030A0006CE286EE95E00E949E2B4C0C5D1C6E1C23
:1030B0007F1C898D9A8DAB8DBC8D84159505A605D9
:1030C000B70520F449885A886B887C88812C912C1C
:1030D000540129893A894B895C89283E334041054E
:1030E000510509F07FCEA296E2E10C94DB2FACE112
:1030F000B0E0EDE7F8E10C94C92F0E94A0296B0124
:103100007C0181E00E94B00A14E703E0198361E0CA
:10311000CE0101960E940D0C009377050E948B0B47
:103120006AEF70E080E090E00E94C329809177050B
:10313000833089F486EE95E00E94A02C892B59F407
:103140000E94A0296C197D098E099F096038734C73
:10315000894C9140D8F280917705833009F44FC0B3
:103160008FE70E94A9090E94BC098983843511F068
:1031700083E05CC00E94BC0910924A0580934B0515
:103180000E94BC0920914A0530914B05280F311D42
:1031900030934B0520934A050E94BC0980934C054F
:1031A0000E94BC0980934D05813110F7F12C0F2D41
:1031B00010E080914D0590E0880F991F08171907BE
:1031C00040F40E94BC09F801E25BFA4F8083F3945B
:1031D000EECF80E7898361E0CE0101960E940D0C5D
:1031E00083E0809377050E948B0B62E370E080E0C0
:1031F00090E00E94C32980917705833011F482E02A
:1032000015C08FE70E94A9090E94BC0989838035F7
:1032100009F0AECF03EA15E00E94BC09F8018193E2
:103220008F01F5E00E3B1F07B9F781E06C96E8E0EF
:103230000C94E52F80914905992787FD9095A92F3A
:10324000B92FFC013196EB30F10508F066C0EC5C5B
:10325000FF4F0C94F62F62E778E086EE95E00E942F
:103260007A2B88E893E00E94620C6AE578E086EEAB
:1032700095E00E947A2B65E378E086EE95E00E9467
:103280007A2B6BE078E086EE95E00E947A2B6AEE6E
:1032900077E086EE95E00E947A2B6DEB77E086EE84
:1032A00095E00E947A2B67E977E086EE95E00E9430
:1032B0007A2B63E777E086EE95E00E947A2B6CE448
:1032C00077E086EE95E00E947A2B86EE95E00E94EC
:1032D000662B0E94A20D21C06FE277E01AC06AE05F
:1032E00077E017C065EF76E014C066ED76E011C0B8
:1032F00062E976E00EC06DE776E00BC068E676E046
:1033000086EE95E00E947A2B62E276E002C06CE0E5
:1033100076E086EE95E00E947A2B6AE070E080E02D
:1033200090E00E94C32986EE95E00E94A02C892B94
:1033300029F086EE95E00E94CD2CF5CF0895ACE102
:10334000B0E0E5EAF9E10C94C92F909149059F3F5F
:1033500009F023C1482F50E0FA013A97EF36F10502
:1033600008F00FC1E15CFF4F0C94F62F61E172E0B1
:10337000A0C06DE172E086EE95E00E948C2B85E79F
:1033800089838BE1E3EAF5E0DE01129601900D926C
:103390008A95E1F76CE1CE0101960E940D0C0E9426
:1033A0008B0B83E08093770568EC70E080E090E021
:1033B0000E94C32980917705843009F0E2C08FE72D
:1033C0000E94A9090E94BC098983853509F0D9C0EA
:1033D0006DEE74E086EE95E00E947A2B6FEC74E05F
:1033E00086EE95E00E947A2B61EB74E096C065E36F
:1033F00072E086EE95E00E948C2B89E6898361E07D
:10340000CE0101960E940D0C0E948B0B83E08093ED
:10341000770568EC70E080E090E00E94C32980911D
:103420007705843009F0ADC08FE70E94A9090E949A
:10343000BC0989838E010E5F1F4F7E014DE1E40EB2
:10344000F11C0E94BC09F80181938F01EE15FF0564
:10345000C1F78BE1FE013296A3EAB5E001900D922F
:103460008A95E1F78981893409F08BC063E974E0BA
:1034700086EE95E00E947A2B65E774E086EE95E093
:103480000E947A2B67E574E048C06FE472E086EE34
:1034900095E00E948C2B8EEF8093490572C080527C
:1034A0008750805390914C05981708F066C06EE5E0
:1034B00072E086EE95E00E948C2B63C084E18093DD
:1034C000490560E274E029C085E18093490569EE11
:1034D00073E023C086E18093490562EB73E01DC071
:1034E00087E18093490568E673E017C088E180931F
:1034F000490567E573E011C089E18093490563E4FC
:1035000073E00BC08AE1809349056EE273E005C069
:103510008BE18093490566E073E086EE95E00E94BA
:103520007A2B2FC06CEE72E086EE95E00E947A2B2B
:103530008091B10591E01DC066ED72E086EE95E0E8
:103540000E947A2B8091B10592E013C061EC72E089
:1035500086EE95E00E947A2B8091B10594E009C037
:1035600066EA72E086EE95E00E947A2B8091B105C2
:1035700098E089278093B1058FEF809349050E94D9
:10358000431086EE95E00E94A02C892B09F45BC1C4
:1035900086EE95E00E94CD2CF4CF0E944211882344
:1035A00009F451C18091E304811104C08FEF80932D
:1035B000490541C140E050E060E070E084EE94E0F5
:1035C0000E946D3040914905042F112707FD109589
:1035D000212F312FF8013197EB31F10508F01BC194
:1035E000E255FF4F0C94F62F552747FD509520913B
:1035F0004C0530E0241735070CF40DC18B019C01FC
:103600000150110921093109003211052105310547
:1036100058F0C0904D05EFE4F5E0F12CD12CA8E274
:10362000EA2E415051090FC0FA01ED55FA4F615091
:103630006083D9C0DF0111972C9130E02417350742
:1036400029F0F3943296FC10F5CFCBC00E2D10E08C
:1036500020E030E0061717072807390741F42081DA
:10366000DA01AD55BA4F11962C93DD24D394E3942F
:10367000E8CF6F3F71058105910511F008F0CBC0CF
:103680006093BB05B0C06F3F71058105910511F0D6
:1036900008F0C1C06093BC05A6C06F3F71058105ED
:1036A000910511F008F0B7C06093BD059CC0209152
:1036B000E40420622037E9F440E050E060E070E08C
:1036C00085EE94E00E946D309B01AC01DC01CB01E2
:1036D0000197A109B1090897A105B10508F0AEC08D
:1036E000A4EDB0E30E94472F6A5E7C4A8A46954E5D
:1036F00024C02636E9F440E050E060E070E085EE5A
:1037000094E00E946D309B01AC01DC01CB0101977C
:10371000A109B1090797A105B10508F08FC0A8EA72
:10372000B1E60E94472F645E7C438E46944E05C0EE
:10373000611571058105910579F08B019C01005C93
:103740001D49284535430130FAE51F07F2E62F07EA
:10375000F2E03F0708F05FC06093B3057093B405D3
:103760008093B5059093B6053EC06F3F7105810506
:10377000910511F008F04FC06093B70534C08B017C
:103780009C0101501109210931090F3F1105210543
:10379000310508F040C06093B80525C08B019C013D
:1037A000045C1940210931090D344DE1140721054C
:1037B000310528F47093BA056093B90514C06115FA
:1037C00071058105910521F48FEF8093B2050BC03F
:1037D0006134710581059105F0F461506093B20583
:1037E00002C0DD20C1F08091E20481111AC08091F5
:1037F000830590918405A0918505B0918605019679
:10380000A11DB11D8093830590938405A093850528
:10381000B093860506C060E772E086EE95E00E94F0
:103820008C2B0E9438118FEF809349056AE086EE59
:1038300095E00E949E2B0E94431005C061E070E05D
:1038400080E090E07ACF6C96E8E00C94E52F6AE592
:1038500072E086EE95E00E947A2B62E472E086EEDA
:1038600095E00E947A2B86EE95E00E94A02C892B91
:1038700031F086EE95E00E94CD2C0E949F190E94A7
:103880007718823029F0833051F46DE072E002C085
:1038900064E272E086EE95E00E947A2B08958FEF45
:1038A000809349051092E2040E94431080914905DB
:1038B0008E3F69F086EE95E00E94A02C892BB1F333
:1038C00086EE95E00E94CD2C0E949F19EFCF0895BF
:1038D0000F931F93109149051F3F09F0D2C08934FF
:1038E00009F457C000F5883309F469C058F48033EF
:1038F00009F477C008F061C08B3109F440C081320F
:10390000B1F1B9C0813409F487C030F4893309F4C6
:1039100066C0803461F1AFC0823409F48EC0863451
:1039200009F448C0A8C0823609F487C078F4883505
:1039300031F128F48235C1F18335E1F09CC08A353C
:1039400009F494C0813609F467C095C0823761F1EB
:1039500028F4863679F18936E1F08DC0883779F020
:103960008A3709F483C0833709F085C003C061E159
:1039700072E015C00E94730D6EE872E004C00E94F0
:103980007C0D68EA72E086EE95E00E948C2B8EEF4B
:1039900070C00E947A060E94BF0667EC72E086EE55
:1039A00095E00E948C2B67C081E00E94DF0660EEEC
:1039B00072E0F5CF0E94ED105EC080535AC06AEFEE
:1039C00071E086EE95E00E947A2B9091A20588E046
:1039D000890F8871977E892B8093A2051AC089E090
:1039E00048C067EE71E086EE95E00E947A2B8091E8
:1039F000C3059091C405A091C505B091C60520E10D
:103A000082278093C3059093C405A093C505B09306
:103A1000C605109349052FC061ED71E086EE95E073
:103A20000E947A2B8091C3059091C405A091C50591
:103A3000B091C60540E4842710C060EC71E086EECA
:103A400095E00E947A2B8091C3059091C405A091C6
:103A5000C505B091C60520E282278093C3059093E7
:103A6000C405A093C505B093C60502C00E94271CDB
:103A70008FEF80934905809149058E3F09F0D4C0AE
:103A8000DDC00E944211882309F4D8C08091E3046C
:103A9000811104C08FEF80934905C6C040E050E01B
:103AA00060E070E084EE94E00E946D300091490582
:103AB000112707FD1095212F312FF8013197E9309B
:103AC000F10508F0B4C0E753FF4F0C94F62F8B01BB
:103AD0009C01015C1D49284535430F3F194522468D
:103AE000324008F0A4C060937F05709380058093F6
:103AF00081059093820577C0609383057093840558
:103B0000809385059093860581E08093E2046BC0E5
:103B1000683071058105910508F089C060938705BB
:103B200062C08B019C0101501109210931090A3041
:103B300011052105310508F07AC06093880553C04E
:103B400061EB71E084EE94E00E94A73110E00097F1
:103B500099F00E948131009779F0183130F4E12F0B
:103B6000F0E0E658FA4F87871F5F61EB71E080E075
:103B700090E00E94A731EBCF1831A8F5E12FF0E0DB
:103B8000E658FA4F17861F5FF7CF6530710581053C
:103B9000910508F04CC06093A10525C08B019C01E4
:103BA000015011092109310906301105210531059E
:103BB000F0F52091A205287F262B2093A20513C0A3
:103BC0008B019C0101501109210931090115124C89
:103BD0002140310560F560937B0570937C058093EF
:103BE0007D0590937E058091E204811113C0809140
:103BF000830590918405A0918505B0918605019675
:103C0000A11DB11D8093830590938405A093850524
:103C1000B09386050E9438118FEF809349056AE0C2
:103C200086EE95E00E949E2B0E941A1907C060E75D
:103C300072E086EE95E00E948C2BECCF1F910F91E5
:103C400008958FEF809349051092E2040E941A199B
:103C5000809149058E3F69F086EE95E00E94A02C88
:103C6000892BB1F386EE95E00E94CD2C0E94681C52
:103C7000EFCF6AE070E080E090E00E94C32986EE1A
:103C800095E00E94A02C892B29F086EE95E00E94F9
:103C9000CD2CF5CF0895CF93C82F682F86EE95E0F1
:103CA0000E94FA2C90916E059C2790936E05CF91FF
:103CB0000895A1E0B0E0EFE5FEE10C94CF2F9983E9
:103CC0000E944B1E9981892F0E944B1E2196E2E093
:103CD0000C94EB2F1F93CF93DF93182FEB011092CF
:103CE0006E0565EB70E086EE95E00E94590662E68F
:103CF00070E086EE95E00E945906812F0E944B1ECF
:103D0000CE010E94591EDF91CF911F9108956091BD
:103D10006E0586EE95E00E94FA2C0895A1E2B0E0CF
:103D2000E4E9FEE10C94CB2F7B018A018C3009F48D
:103D300053C108F040C0863009F4BCC018F5833088
:103D400009F491C070F4813009F472C0823009F036
:103D50004AC26BE170E082E00E946A1E03EA15E04D
:103D600078C0843009F487C0853009F03CC2609186
:103D70004D0570E0660F771F85E00E946A1E0EE415
:103D800015E086C0893009F4A7C070F4873009F4C3
:103D90009BC0883009F027C261E070E088E00E9493
:103DA0006A1E8091D80525C28A3009F4CAC08B30BA
:103DB00009F4F2C018C28A3609F475C1D8F48736FE
:103DC00009F43AC138F4853609F40EC1863609F48F
:103DD0001FC109C2883609F437C1893609F003C208
:103DE00061E070E089E60E946A1E0E947A060E94E5
:103DF000BF06F7C18D3609F4D4C138F48B3609F407
:103E000091C18C3609F49AC1EEC18E3609F4DEC137
:103E1000873C09F0E8C161E070E087EC0E946A1E0F
:103E200081E00E944B1E0E94871E10926F05E5C123
:103E300069E270E081E00E946A1E0AE715E0F8017D
:103E400081918F010E944B1EF5E0033A1F07B9F7DD
:103E5000D2C1F80181918F010E944B1EF5E00E3B0B
:103E60001F07B9F7C8C161E070E083E00E946A1ED5
:103E70000E947718BEC161E070E084E00E946A1E73
:103E800081E00E944B1E0E94871E0E94AA16B5C1A7
:103E900080914D0590E0880F991F98012E54354070
:103EA0002817390708F0A7C1F80181918F010E94F6
:103EB0004B1EEECF62E070E086E00E946A1E88E84A
:103EC00093E00E94591E97C161E070E087E00E9474
:103ED0006A1E80914C058DC186E6898361E0CE0122
:103EE00001960E940D0C0E948B0B83E08093770556
:103EF00068EC70E080E090E00E94C3298091770533
:103F00008430D9F48FE70E94A9090E94BC098983F3
:103F1000863469F460E270E089E00E946A1E10E273
:103F20000E94BC090E944B1E1150D1F764C161E090
:103F300070E089E00E946A1E54C161E070E089E08F
:103F400055C169E170E08AE00E946A1E82E08093B8
:103F5000BE05209176058091C3059091C405A0917E
:103F6000C505B091C605222311F0806801C08F7786
:103F70008093C3059093C405A093C505B093C6056F
:103F80000EEB15E0F80181918F010E944B1EF5E0C8
:103F9000073D1F07B9F72FC161E270E08BE00E9477
:103FA0006A1E8091AA048F3F39F08091AA0491E0A3
:103FB000980F9093AA0402C08091AA040E944B1EFD
:103FC00010E0812F0E9437160E943C090E94591E62
:103FD0001F5F1031B1F70FC161E070E08CE00E940B
:103FE0006A1E8091D70505C161E070E085E60E94F8
:103FF0006A1E89E2E816F10409F0FAC0D801EAE77E
:10400000F5E08D91819385E0E33AF807D1F7E9C0B7
:1040100061E070E086E60E946A1EEBE1EE16F104B4
:1040200009F0E6C0D801E3EAF5E08D91819385E0DF
:10403000EE3BF807D1F7D5C061E070E087E60E945B
:104040006A1E0E94730DCDC061E070E088E60E9498
:104050006A1E85E789838BE1E3EAF5E0DE011296CB
:1040600001900D928A95E1F76CE1CE0101960E94D4
:104070000D0C0E948B0B83E08093770560E273E068
:1040800080E090E00E94C32980917705843009F098
:10409000AFC08FE70E94A9090E94BC0989838535BA
:1040A00009F0A6C09EC061E070E08AE60E946A1E28
:1040B00089E6898361E0CE0101960E940D0C0E9481
:1040C0008B0B83E08093770560E273E080E090E003
:1040D0000E94C32980917705843009F089C08FE759
:1040E0000E94A9090E94BC0989838E010E5F1F4F9F
:1040F0007E01EDE1EE0EF11C0E94BC09F8018193F6
:104100008F01EE15FF05C1F78BE1FE013296A3EAA0
:10411000B5E001900D928A95E1F78981893409F023
:1041200067C05FC061E070E08BE60E946A1EF80124
:1041300080818093D8050E947C0D53C061E070E0BF
:104140008CE60E946A1EF0E2EF16F10461F487E645
:10415000898380E2F801DE01129601900D928A9522
:10416000E1F761E203C087E4898361E0CE01019653
:104170000E940D0C0E948B0B83E0809377056CE40A
:1041800074E080E090E00E94C3298091770584303C
:1041900079F58FE70E94A9090E94BC09873441F58F
:1041A00020C061E070E08DE60E946A1E89E1E81699
:1041B000F104F1F4D801EEEBF5E08D91819385E007
:1041C000E73DF807D1F70E94C1130BC061E070E032
:1041D0008EE60E946A1EF80180818093D7050E94B6
:1041E0005D0D81E006C061E070E08AEC0E946A1E0D
:1041F00080E00E944B1E0E94871EA196E6E00C9470
:10420000E72FA0E0B0E0E7E0F1E20C94C92FCAECA0
:10421000D3E014E606E035E0F32E44E0E42E53E06C
:10422000D52E62E0C62E86EE95E00E94A02C892B4A
:1042300009F49BC086EE95E00E94CD2C282F809338
:1042400035044091340450E04730510560F7FA01DD
:10425000EE52FF4F0C94F62F853B29F781E08093B7
:104260003404E1CF823609F07DC0C0923404DBCF44
:104270008093330480933204D0923404D4CF9C01D1
:1042800033273093310420933004909132049827DF
:1042900090933204E0923404C6CF382F2227409105
:1042A000300450913104242B352B3093310420936A
:1042B000300490913204982790933204F0923404A1
:1042C0002536310508F4AFCF61E070E08CEC0E9438
:1042D0006A1E81E00E944B1E0E94871E43C02091EF
:1042E0002E0430912F04F901E653FC4F8083909106
:1042F0003204982790933204C901019690932F04B9
:1043000080932E042091300430913104821793075A
:1043100008F489CF0093340486CF8091320482134D
:104320000BC060912E0470912F044AEC53E08091F1
:1043300033040E948E1E0DC062E070E08BEC0E9480
:104340006A1E809133040E944B1E80916E050E946C
:104350004B1EFE01812F11928A95E9F710922F04CE
:1043600010922E04109234045ECFCDB7DEB7E8E091
:104370000C94E52F81E080936F0580916F05882371
:1043800049F086EE95E00E94A02C892BB1F30E94A3
:104390000121F3CF0895AAE2B0E0E1EDF1E20C943F
:1043A000C72F0E9494296B017C0181E00E94B00A12
:1043B00086EE95E00E94A02C892B29F086EE95E0F0
:1043C0000E94CD2CF5CF4398299811E072E6B72EC4
:1043D000E9E2AE2E03E00E9494296C197D098E0952
:1043E0009F09693C710581059105F0F11123E1F107
:1043F0000E9494296B017C0185B1846285B980EDAE
:1044000097E00E94B607B982EAE7F5E0DE0112966E
:104410008A2D01900D928A95E1F76AE2CE0101960C
:104420000E940D0C85B18B7D85B980E090E00E94E3
:10443000B607009377050E948B0B62E370E080E083
:1044400090E00E94C32980917705843061F4009345
:1044500077058FE70E94A9090E94BC0911E0823408
:1044600019F410E001C011E087E00E94B92A892BFD
:10447000B1F411E014C0439A299A85B1846285B9D8
:1044800086EE95E00E94CD2C8D309105C1F074F43C
:104490000A97A9F04398299885B18B7D85B986EE56
:1044A00095E00E94A02C892B31F795CF833291059E
:1044B00079F08234910571F70E94BA21EBCF62EB5B
:1044C00071E086EE95E00E947A2B0E94211EE2CFD9
:1044D0000E94AA16DFCF8F929F92AF92BF92CF9287
:1044E000DF92EF92FF921F93CF93DF9387E00E94BA
:1044F000B92A892B09F089C068EC70E080E090E06F
:104500000E94C32980E090E00E94B6070E9494298F
:104510004B015C016B017C0180ECC80E82E1D81E6E
:10452000E11CF11C0E9494296C157D058E059F05E8
:1045300030F487E00E94B92A892BA1F364C087E098
:104540000E94B92A892B09F05EC080ED97E00E9495
:10455000B6070E9494296B017C01D0E0C1E088E499
:10456000880E86E2981EA11CB11C11E087E00E9413
:10457000B92A892B21F58C149D04AE04BF0430F4B4
:1045800080ED97E00E94B607D1E0F0CF0E94942919
:104590006C197D098E099F09693C7105810591059A
:1045A00028F30E9494296B017C01C12719F080ED4A
:1045B00097E002C080E090E00E94B607D7CF80E08D
:1045C00090E00E94B607DD23B9F08091D70590E016
:1045D000019665E070E00E946A2F8093D7050E94E3
:1045E0005D0D0E94DC130E947C0D64EF71E080E0A1
:1045F00090E00E94C32909C080E00E94DF060E946B
:10460000F4110E94730D0E94CB21DF91CF911F9175
:10461000FF90EF90DF90CF90BF90AF909F908F90E2
:104620000895CF92DF92EF92FF9280E00E940D08F2
:104630000E94E40761E081E10E944D2A61E08DE083
:104640000E944D2A61E089E00E944D2A61E08AE0E3
:104650000E944D2A60E087E00E944D2A60E08BE0D6
:104660000E944D2A61E08BE00E94862A60E08CE087
:104670000E944D2A61E08CE00E94862A60E088E07A
:104680000E944D2A61E088E00E94862A0E949F07CE
:1046900040E052EC61E070E086EE95E00E94E82D8B
:1046A0000E94DC130E947C0D0E94C1138FEF809347
:1046B000AA040E94F90778940E9494296B017C0156
:1046C0008091AA048F3F59F40E9494296C197D09A6
:1046D0008E099F09603D77408105910588F380ED43
:1046E00097E00E94B60761E087E00E94862A439A1D
:1046F000299A86EE95E00E94A02C892B29F086EE5F
:1047000095E00E94CD2CF5CF6DEF72E086EE95E03E
:104710000E945B2B88E893E00E94620C64E173E0E6
:1047200086EE95E00E945B2B4AE050E063E070E08B
:1047300086EE95E00E942B2C62E370E080E090E032
:104740000E94C32986EE95E00E94A02C04970CF1EC
:1047500086EE95E00E94CD2C82349105D1F486EE50
:1047600095E00E94CD2C8E34910599F486EE95E06B
:104770000E94CD2C8434910561F486EE95E00E9470
:10478000CD2C819731F480E090E00E94B6070E9422
:10479000CB2140917B0550917C0560917D05709106
:1047A0007E05DB01CA010197A109B1090497A105A2
:1047B000B10590F44093A904433051F42EE240EA4D
:1047C00056E861E070E086EE95E00E94692E08C030
:1047D00040E052EC61E070E086EE95E00E94E82D4A
:1047E0000E946B224398299880E090E00E94B607CF
:1047F0000E94C1131092C9048091C30583FF11C0A8
:1048000080918F05882351F080919605882331F09F
:1048100080919D05882311F087E001C085E0809399
:10482000C90480E00E94B00A8091CA040E94E40991
:104830000E948B0B10923F0410923E0410923D0494
:10484000F12C8091D8058F15B0F062E370E080E024
:1048500090E00E94C32980ED97E00E94B60762E3D2
:1048600070E080E090E00E94C32980E090E00E9428
:10487000B607F394E6CF8091A20584FF08C0982F75
:10488000987181E0983109F080E00E94B0118FE0CA
:104890000E940D08FF90EF90DF90CF900895EF9267
:1048A000FF920F931F93CF93DF938C016EE770E01D
:1048B00086EE95E00E945906E801F12CF0E2EF2E19
:1048C0008E0188818D57823048F46DE770E086EE66
:1048D00095E00E94590688818E2588832196F801EB
:1048E000608186EE95E00E94FA2CF394F9E0FF12C5
:1048F000E7CF6EE770E086EE95E00E945906CDB7EF
:10490000DEB7E6E00C94E72FA9E0B0E0EAE8F4E2D5
:104910000C94CF2F9091CB0491110EC09EEF9983F0
:104920008A836B8350E0559547954C832D83198678
:1049300018861F821E822EC04091D004842F90E0E2
:10494000B4E095958795BA95E1F7242F2F7030E064
:104950008217930719F18DEF89831B82FE0134962C
:1049600050E0842F90E0A4E095958795AA95E1F713
:10497000242F2F7030E08217930749F0DC01AF52EB
:10498000BB4F8C918193405F5F5F563051F74093EE
:10499000D0045A83CE0101960E944F248091CB040B
:1049A00090E0019666E070E00E946A2F8093CB044D
:1049B0002996E2E00C94EB2FA0E0B0E0E2EEF4E206
:1049C0000C94C82F6C016EE770E086EE95E00E94B3
:1049D00059068601E12CF12CC0E0D0E030E2B32E84
:1049E000F801608183E8860F823078F46DE770E02B
:1049F00086EE95E00E945906F80160816B2570E013
:104A000086EE95E00E94590604C086EE95E00E946D
:104A1000FA2CE114F10459F0F80180819E01280F6D
:104A2000311DC901C92FDD27C80FD91FDD273FEF71
:104A3000E31AF30A89E0E816F10459F028E0E216D7
:104A4000F10421F48C2F8095F60180870F5F1F4FB2
:104A5000C7CFCDB7DEB7E9E00C94E42FA9E0B0E012
:104A6000E4E3F5E20C94CF2FE82F362F8091CB04AE
:104A700090E0019664E270E00E946A2F8093CB047C
:104A800058E9598350E15A83813089F048F08230E7
:104A9000B9F08330D9F48B8381EF8C833D8319C0C7
:104AA00085E08B8381EF8C832F5F2D8312C08B83F6
:104AB00081EF8C8384E6489FA00111245D8309C0A7
:104AC00084E08B8381EF8C83ED8303C00E94ED1122
:104AD00004C0CE0101960E94DC242996E2E00C94E9
:104AE000EB2FA2E0B0E0E7E7F5E20C94C42F182F1B
:104AF000762E2A8349830E94A0296B017C01809134
:104B0000E1048090CC049090CD04A090CE04B090AD
:104B1000CF042A8149818823C1F0D701C6018819B1
:104B20009909AA09BB094C015D0191EE89169EE223
:104B30009906A104B10420F1241708F4422F202F74
:104B4000672D812F0E942E2513C0D701C601881919
:104B50009909AA09BB094C015D0191E3891695E702
:104B60009906A104B10460F0672D812F0E9484246E
:104B7000C092CC04D092CD04E092CE04F092CF0447
:104B80002296EDE00C94E02FA2E2B0E0EAECF5E230
:104B90000C94C52F8CE00E94CB0981110FC06CE1F1
:104BA00073E086EE95E00E948C2B439A299A80E070
:104BB0000E94B00A0E948B0B4398299886EE95E0DC
:104BC0000E94A02C892B01F186EE95E00E94CD2C4D
:104BD0009091A904992319F00E941814EFCF4091E5
:104BE0003E0450E09A012F5F3F4F2F7133276091B1
:104BF0003F0470E02617370709F3FA01E75BFB4F24
:104C0000808320933E04DACF80917705843009F0C9
:104C100086C00E94A029611571058105910549F0A2
:104C20006093BB047093BC048093BD049093BE0456
:104C30000CC081E090E0A0E0B0E08093BB049093D2
:104C4000BC04A093BD04B093BE048091AD049091C8
:104C5000AE0481609093AE048093AD0483E08093B2
:104C600077058FE70E94A90909E614E00E94BC09B4
:104C7000F80181938F01F4E002371F07B9F7209103
:104C8000720480916904982F922796FF3BC090E4AC
:104C9000922790937204982F98739833F1F410E050
:104CA000212F30E080916904877090E0821793078C
:104CB0004CF11F5F2091A205812F90E0FC01E75984
:104CC000FB4F24FF04C080810E94CF11E9CF608197
:104CD00086EE95E00E94FA2CE3CF8F7399F48091D1
:104CE0006A048093B60480916B048093B40480912D
:104CF0006C048093B30480916F0490E09093AC04B3
:104D00008093AB0480913D04813019F482E080935C
:104D10003D0480913D04833011F410923D040E94C3
:104D2000A0296B017C018091AF049091B004A09107
:104D3000B104B091B2040097A105B105C9F0A70173
:104D40009601281B390B4A0B5B0BDA01C901883B22
:104D50009B40A105B10560F00E94FA098093B5045B
:104D60001092AF041092B0041092B1041092B204E9
:104D70008091BF049091C004A091C104B091C2047D
:104D800046015701881A990AAA0ABB0A8AE795E0E0
:104D90000E94270886169706A806B90608F4B3C02D
:104DA000C092BF04D092C004E092C104F092C20449
:104DB0000E9457068091AA048830A0F08091C30514
:104DC0009091C405A091C505B091C6055CE1B6956A
:104DD000A795979587955A95D1F7892B8A2B8B2B79
:104DE00009F0CCC18091AA048F5F8093AA048091BE
:104DF000BB049091BC04A091BD04B091BE04009787
:104E0000A105B105F1F0C81AD90AEA0AFB0A8AE736
:104E100095E00E9427086C157D058E059F0508F01A
:104E20001FC18091C30584FD04C080ED97E00E94FE
:104E3000B6071092BB041092BC041092BD041092ED
:104E4000BE0490917204907C9093720450913E0441
:104E500080913F0420913D04581709F41EC122306F
:104E600009F01BC1905890937204E091A205E7707D
:104E7000F0E0E658FC4F6081693008F0F6C0615000
:104E800040E04613F4C080933F0487E3840F909181
:104E90007204892B809372044093400483E08093D2
:104EA0003D0485B1846285B9109187058091C9045C
:104EB000811142C18091C30582FD4AC1812F0E94A8
:104EC000AB0A8091CA040E94E409E091A205E77050
:104ED000F0E0E658FC4F608182E794E00E94C60B48
:104EE0008091C30582FD3EC1E091CA04EF5FE0936B
:104EF000CA04E83109F43FC1F0E0E658FA4F87856B
:104F0000882309F438C10E94350C813069F58091FD
:104F1000A205887149F18091AD049091AE04880F8B
:104F2000991F9093AE048093AD0483E0809377053E
:104F30000E948B0B0E94A0296093AF047093B00471
:104F40008093B1049093B204672B682B692B61F4B2
:104F500081E090E0A0E0B0E08093AF049093B004D3
:104F6000A093B104B093B2048091A20584FF2BC03A
:104F70008091BB049091BC04A091BD04B091BE048B
:104F8000892B8A2B8B2BF9F08091AD049091AE0484
:104F90008E7F0E945D09182F6091AB048091B6044A
:104FA0000E940E14482F612F8091B50449A30E94DE
:104FB0000E140091D805282F49A16091B304809167
:104FC000B4040E94712585B18B7D85B98091C70499
:104FD0008130C1F018F08230B1F1DEC087E00E946C
:104FE000B92A892B09F0D8C081E08093C7040E94B8
:104FF00094296093C3047093C4048093C504909370
:10500000C604CAC087E00E94B92A892B31F50E94E4
:105010009429C090C304D090C404E090C504F090DB
:10502000C6046C197D098E099F09693E734081058C
:10503000910508F4B1C082E08093C70480ED97E049
:105040000E94B607A9C087E00E94B92A892B09F4FB
:10505000A3C080E090E00E94B6071092C7049CC0F5
:1050600080E090E00E94B607ECCE68E009CF85179B
:1050700009F409CF4F5F242F30E090E0F901EE589A
:10508000FB4FDC01A75BBB4F7C917083F901E05CB7
:10509000FB4F708301968F71F4CE2430B1F42091D0
:1050A000400481E494E0A3E7B4E0FC013E2F381B08
:1050B000321718F431913D93F9CF87E3820F909125
:1050C0007204892B80937204E9CE8091C7048230E8
:1050D00059F4916090937204439A299A8E010F5F5C
:1050E0001F4FF12CB80111C04398299880913D04BD
:1050F000811103C081E080933D0480913D048330A1
:1051000069F784E080933D04E9CF8F2D69A37AA3EA
:105110000E943716F801819391938F01F39469A14E
:105120007AA1F0E1FF12F1CF8091A20543E754E0AC
:1051300087700E94AC08B5CE112309F4BBCE9091C4
:10514000C80421E0290F2093C8049813B3CE20C0CF
:105150008BE00E94B92A892B09F0B0CE439A299A94
:1051600017E0ACCE8BE00E94B92A892B09F0BCCEA7
:1051700043982998B9CE1092CA04C5CE8091AA044A
:10518000883011F4439A299A89E08093AA04BBCE0F
:105190001092C80411508ECEA296ECE00C94E12F30
:1051A0008230E8F4E82FF0E0EE0FFF1FE752FA4FED
:1051B00071836083813041F0809169008C7F842B02
:1051C00080936900E89A089580916900440F551F03
:1051D000440F551F837F842B80936900E99A0895BB
:1051E0001F920F920FB60F9211242F933F934F935C
:1051F0005F936F937F938F939F93AF93BF93EF933F
:10520000FF938091D9059091DA05892B29F0E091DF
:10521000D905F091DA050995FF91EF91BF91AF9112
:105220009F918F917F916F915F914F913F912F91BE
:105230000F900FBE0F901F9018951F920F920FB6F0
:105240000F9211242F933F934F935F936F937F930C
:105250008F939F93AF93BF93EF93FF938091DB0561
:105260009091DC05892B29F0E091DB05F091DC05BC
:105270000995FF91EF91BF91AF919F918F917F9190
:105280006F915F914F913F912F910F900FBE0F90B3
:105290001F9018951F920F920FB60F9211242F9303
:1052A0003F938F939F93AF93BF938091DE0590912F
:1052B000DF05A091E005B091E1053091DD0523E027
:1052C000230F2D3720F40196A11DB11D05C026E83E
:1052D000230F0296A11DB11D2093DD058093DE05ED
:1052E0009093DF05A093E005B093E1058091E2057E
:1052F0009091E305A091E405B091E5050196A11D0B
:10530000B11D8093E2059093E305A093E405B0936B
:10531000E505BF91AF919F918F913F912F910F9094
:105320000FBE0F901F9018952FB7F8946091DE056F
:105330007091DF058091E0059091E1052FBF089500
:105340003FB7F8948091E2059091E305A091E405C0
:10535000B091E50526B5A89B05C02F3F19F0019631
:10536000A11DB11D3FBF6627782F892F9A2F620F8D
:10537000711D811D911D42E0660F771F881F991FC7
:105380004A95D1F70895CF92DF92EF92FF92CF9393
:10539000DF936B017C010E94A029EB01C114D104B1
:1053A000E104F10479F00E94A0296C1B7D0B683E9A
:1053B0007340A0F381E0C81AD108E108F108C85190
:1053C000DC4FECCFDF91CF91FF90EF90DF90CF904B
:1053D0000895789484B5826084BD84B5816084BD6D
:1053E00085B5826085BD85B5816085BDEEE6F0E05E
:1053F000808181608083E1E8F0E0108280818260BA
:105400008083808181608083E0E8F0E0808181603A
:105410008083E1EBF0E0808184608083E0EBF0E06A
:10542000808181608083EAE7F0E08081846080830E
:1054300080818260808380818160808380818068B8
:1054400080831092C1000895833081F028F4813068
:1054500099F08230A1F008958630A9F08730B9F034
:105460008430D1F4809180008F7D03C080918000D2
:105470008F7780938000089584B58F7702C084B5BC
:105480008F7D84BD08958091B0008F7703C0809197
:10549000B0008F7D8093B0000895CF93DF9390E0AC
:1054A000FC01ED50F44F2491FC01E95FF34F84912E
:1054B000882349F190E0880F991FFC01E15DF34FCB
:1054C000A591B4918B5D934FFC01C591D4919FB789
:1054D000611108C0F8948C91209582238C93888167
:1054E00082230AC0623051F4F8948C91322F3095A7
:1054F00083238C938881822B888304C0F8948C91B9
:10550000822B8C939FBFDF91CF910895A1E0B0E0F3
:10551000ECE8FAE20C94CD2F282F30E0F901E152AB
:10552000F44F8491F901ED50F44F1491F901E95FC2
:10553000F34F04910023C9F0882321F069830E946E
:10554000242A6981E02FF0E0EE0FFF1FEB5DF34F9F
:10555000A591B4919FB7F8948C91611103C01095F7
:10556000812301C0812B8C939FBF2196E4E00C9492
:10557000E92FCF93DF93282F30E0F901E152F44F68
:105580008491F901ED50F44FD491F901E95FF34FA3
:10559000C491CC2391F081110E94242AEC2FF0E0D9
:1055A000EE0FFF1FE55EF34FA591B4912C912D23D3
:1055B00081E090E021F480E002C080E090E0DF91A3
:1055C000CF9108958E3008F08E50877020919D0104
:1055D00090E4299F90011124822B80937C0080917C
:1055E0007A00806480937A0080917A0086FDFCCFF7
:1055F000809178002091790090E0922B0895A0E0AE
:10560000B0E0E5E0FBE20C94C92F6C017A01EB01FC
:10561000E60EF71E00E010E0CE15DF0561F069919F
:10562000D601ED91FC910190F081E02DC601099524
:10563000080F191FF1CFC801CDB7DEB7E8E00C9411
:10564000E52F6115710589F0DB010D900020E9F768
:10565000AD0141505109461B570BDC01ED91FC9106
:105660000280F381E02D0995089580E090E008958F
:10567000EF92FF920F931F93CF93DF938C01FB0167
:10568000C0E0D0E064917F018FEFE81AF80A66234A
:1056900061F0D801ED91FC910190F081E02DC801FD
:1056A0000995C80FD91FF701EDCFCE01CDB7DEB7F1
:1056B000E6E00C94E72F0E94212B0895DC01ED9188
:1056C000FC910190F081E02D099508950F931F93AF
:1056D000CF93DF93EC016DE00E945E2B8C016AE0BA
:1056E000CE010E945E2B800F911FDF91CF911F9101
:1056F0000F9108950F931F93CF93DF93EC010E94B6
:10570000382B8C01CE010E94662B800F911FDF91F8
:10571000CF911F910F9108950F931F93CF93DF9314
:10572000EC010E94212B8C01CE010E94662B800F80
:10573000911FDF91CF911F910F9108950F931F93A8
:10574000CF93DF93EC010E945E2B8C01CE010E946F
:10575000662B800F911FDF91CF911F910F910895BC
:10576000A1E2B0E0E6EBFBE20C94C52F7C01C42E75
:10577000E52FCB01D22E19A221E02D1510F02AE041
:10578000D22E8E010F5D1F4F8D2C912CA12CB12C90
:105790006C2D7E2FA50194010E947E2F8C2DD29E10
:1057A00080191124015011098A3010F4805D01C064
:1057B000895CF8018083211531054105510521F0EF
:1057C000C22EE32FCA01E4CFB801C7010E94212BEA
:1057D000A196ECE00C94E12FA0E0B0E0E2EFFBE258
:1057E0000C94C92FEC016A017B012115310541F4AC
:1057F000E881F9810190F081E02D642F09951DC0A9
:105800002A303105A9F477FF12C06DE20E945E2BA9
:105810008C0144275527BA014C195D096E097F098F
:105820002AE0CE010E94B02B800F911F06C02AE013
:10583000B701A601CE010E94B02BCDB7DEB7E8E0DC
:105840000C94E52F9A01AB01662757FD6095762FE2
:105850000E94EC2B08950F931F93CF93DF93EC01DD
:105860009A01AB01662757FD6095762F0E94EC2BBD
:105870008C01CE010E94662B800F911FDF91CF918A
:105880001F910F9108952115310549F4DC01ED9127
:10589000FC910190F081E02D642F099508950E94FC
:1058A000B02B08959A01462F50E060E070E00E940E
:1058B000432C08959A01AB0160E070E00E94432CF4
:1058C00008950F931F93CF93DF93EC010E94432C15
:1058D0008C01CE010E94662B800F911FDF91CF912A
:1058E0001F910F9108950F931F93CF93DF93EC01B6
:1058F0009A01AB0160E070E00E94432C8C01CE0164
:105900000E94662B800F911FDF91CF911F910F9105
:1059100008950F931F93CF93DF93EC019A01462FC5
:1059200050E060E070E00E94432C8C01CE010E94A8
:10593000662B800F911FDF91CF911F910F910895DA
:10594000FC0124853585F901E05CFF4F8081918160
:10595000F901EE5BFF4F20813181821B930B8F7326
:1059600099270895FC0184859585FC01E05CFF4F33
:1059700040815181FC01EE5BFF4F20813181421754
:10598000530741F00190F081E02DE80FF91F80816D
:1059900090E008958FEF9FEF0895FC018485958531
:1059A000FC01E05CFF4F40815181FC01EE5BFF4F49
:1059B000208131814217530779F0A081B181A80F6E
:1059C000B91F8C91208131812F5F3F4F2F73332777
:1059D0003183208390E008958FEF9FEF0895FC01BD
:1059E00081A1882329F0A489B5898C9186FFFBCFFA
:1059F00011A20895CF93DF93FC0126853785D90145
:105A0000A05CBF4F8D919C91119701968F73992740
:105A1000E901CE5BDF4F4881598184179507D9F39F
:105A20000D90BC91A02DA20FB31F6C93A685B785D6
:105A3000A05CBF4F11969C938E93A689B7892C9139
:105A400081E090E0078C02C0880F991F0A94E2F76A
:105A5000282B2C9381E081A30488F589E02D808197
:105A60008064808381E090E0DF91CF910895089574
:105A70001F920F920FB60F9211242F933F934F93C3
:105A80008F939F93EF93FF938091C00082FD1CC082
:105A90004091C60080918C0690918D0601968F737F
:105AA000992720918E0630918F068217930771F007
:105AB000E0918C06F0918D06E45BF94F4083909362
:105AC0008D0680938C0602C08091C600FF91EF91F5
:105AD0009F918F914F913F912F910F900FBE0F90FB
:105AE0001F90189586EE95E00E94A02C892B11F04E
:105AF0000E94372D08951F920F920FB60F92112416
:105B00002F933F938F939F93EF93FF93209148069A
:105B10003091490680914A0690914B062817390723
:105B200031F48091C1008F7D8093C10014C0E09159
:105B30004A06F0914B06E85FF94F208180914A06B2
:105B400090914B0601968F73992790934B06809303
:105B50004A062093C600FF91EF919F918F913F914C
:105B60002F910F900FBE0F901F901895A0E0B0E0FE
:105B7000ECEBFDE20C94C52FFC011382128288EE3F
:105B800093E0A0E0B0E084839583A683B7838CEB99
:105B900093E0918380837587648757874687318B2D
:105BA000208B138B028BF58AE48AD78AC68AB18E42
:105BB000A08E938E828E8F85848F8889858F898928
:105BC000868F8A89878F8B8980A3ECE00C94E12FE4
:105BD000CF92DF92EF92FF92CF93DF93EC016A01B5
:105BE0007B01411581EE580761057105F9F0EC89DB
:105BF000FD8981E090E008A002C0880F991F0A94F7
:105C0000E2F7808360E079E08DE390E0A701960100
:105C10000E947E2F2150310941095109569547951F
:105C200037952795211580E1380798F0EC89FD8993
:105C3000108260E874E88EE190E0A70196010E946E
:105C40007E2F2150310941095109569547953795C5
:105C50002795E889F9893083EA89FB89208319A28D
:105C6000EE89FF89408181E090E09C010C8C02C0AC
:105C7000220F331F0A94E2F7422B4083EE89FF89FB
:105C800040819C010D8C02C0220F331F0A94E2F761
:105C9000422B4083EE89FF8940819C010E8C02C01B
:105CA000220F331F0A94E2F7422B4083EE89FF89CB
:105CB00020810F8C02C0880F991F0A94E2F780950B
:105CC00082238083DF91CF91FF90EF90DF90CF9080
:105CD0000895BF92CF92DF92EF92FF92CF93DF931E
:105CE000EC016A017B01B22E411581EE5807610576
:105CF0007105F9F0EC89FD8981E090E008A002C00F
:105D0000880F991F0A94E2F7808360E079E08DE3C1
:105D100090E0A70196010E947E2F21503109410990
:105D200051095695479537952795211580E13807F4
:105D300098F0EC89FD89108260E874E88EE190E0CB
:105D4000A70196010E947E2F215031094109510976
:105D50005695479537952795E889F9893083EA89DB
:105D6000FB892083E88DF98DB082EE89FF8940811F
:105D700081E090E09C010C8C02C0220F331F0A943A
:105D8000E2F7422B4083EE89FF8940819C010D8C14
:105D900002C0220F331F0A94E2F7422B4083EE89A0
:105DA000FF8940819C010E8C02C0220F331F0A9490
:105DB000E2F7422B4083EE89FF8920810F8C02C0DD
:105DC000880F991F0A94E2F7809582238083DF91E0
:105DD000CF91FF90EF90DF90CF90BF9008958F927A
:105DE0009F92AF92BF92CF92DF92EF92FF920F936A
:105DF0001F9381E08F9385E08F9387E08F9383E0FB
:105E00008F9384E08F93E6EC8E2E912CF2ECAF2EE4
:105E1000B12CA1ECCA2ED12CB0ECEB2EF12C04EC61
:105E200010E025EC30E048E056E06CE476E086EEE9
:105E300095E00E94B62D0F900F900F900F900F904D
:105E40001F910F91FF90EF90DF90CF90BF90AF9098
:105E50009F908F9008950E94E9290E941123C2E724
:105E6000DDE20E94C4252097E1F30E94722DF9CF54
:105E7000A29FB001B39FC001A39F700D811D11248B
:105E8000911DB29F700D811D1124911D08950E94D6
:105E9000382FA59F900DB49F900DA49F800D911D4C
:105EA00011240895B7FF0C94472F0E94472F821B9F
:105EB000930B0895DB018F939F930E94472FBF910F
:105EC000AF91A29F800D911DA39F900DB29F900D49
:105ED0001124089597FB072E16F4009407D077FD40
:105EE00009D00E94FC2F07FC05D03EF490958195C7
:105EF0009F4F0895709561957F4F0895A1E21A2EE6
:105F0000AA1BBB1BFD010DC0AA1FBB1FEE1FFF1F5D
:105F1000A217B307E407F50720F0A21BB30BE40BAD
:105F2000F50B661F771F881F991F1A9469F76095F4
:105F30007095809590959B01AC01BD01CF010895AE
:105F4000052E97FB1EF400940E94B72F57FD07D033
:105F50000E947E2F07FC03D04EF40C94B72F50956F
:105F60004095309521953F4F4F4F5F4F0895909545
:105F70008095709561957F4F8F4F9F4F08952F9219
:105F80003F924F925F926F927F928F929F92AF92C9
:105F9000BF92CF92DF92EF92FF920F931F93CF9316
:105FA000DF93CDB7DEB7CA1BDB0B0FB6F894DEBFAD
:105FB0000FBECDBF09942A88398848885F846E84D3
:105FC0007D848C849B84AA84B984C884DF80EE801D
:105FD000FD800C811B81AA81B981CE0FD11D0FB626
:105FE000F894DEBF0FBECDBFED010895EE0FFF1F89
:105FF0000590F491E02D0994AA1BBB1B51E107C049
:10600000AA1FBB1FA617B70710F0A61BB70B881F48
:10601000991F5A95A9F780959095BC01CD010895D7
:106020008F929F92AF92BF92CF92DF92EF92FF92A8
:10603000CF93DF93EC01688179818A819B8161151F
:1060400071058105910521F464E279ED8BE597E016
:106050002DE133EF41E050E00E94A02F49015A01A9
:106060009B01AC01A7EAB1E40E94472F6B017C01C0
:10607000ACEEB4EFA50194010E94552FC60ED71EB9
:10608000E81EF91EF7FE06C081E0C81AD108E10833
:1060900080E8F80AC882D982EA82FB82C701B60189
:1060A0009F77DF91CF91FF90EF90DF90CF90BF90DF
:1060B000AF909F908F9008950E941030089586E0D1
:1060C00091E00E94103008956093060170930701DB
:1060D000809308019093090108952F923F925F9257
:1060E0006F927F928F929F92AF92BF92CF92DF92E8
:1060F000EF92FF920F931F93CF93DF938B01EA01EF
:106100006115710521F0DB018C9311969C9320970A
:1061100039F09E01225031092332310508F0D8C0F0
:106120007C016701BFEFCB1ADB0A5601F7016080E3
:10613000862D90E00E949F31892B11F07601F1CFDE
:10614000FDE26F120AC0570182E0A80EB11CD70110
:1061500011966C90772473940BC0BBE26B1207C04E
:106160005701E2E0AE0EB11CD70111966C90712C74
:10617000CE018F7E892B89F4B0E36B1237C0F50115
:1061800080818F7D8835D1F46180F2E0AF0EB11C43
:10619000872D8260782EC0E1D0E0CA30D10551F160
:1061A000C031D10521F0C830D10599F409C0CC2403
:1061B000CA94DC2CEC2CAFE0FA2E22C0209769F7B1
:1061C000C8E0D0E0CC24CA94DC2CEC2CFFE1FF2EFC
:1061D00017C06FEF7FEFCB019E01442737FD40953D
:1061E000542F0E947E2F69017A010AC02097A9F6D8
:1061F000CAE0D0E0E9E9CE2EDC2CEC2CE9E1FE2E61
:10620000F50160E020E030E0A9014E01AA2497FCEE
:10621000A094BA2C1F0170ED572E560CA9E0A515BD
:1062200070F48FEB860D8A3118F499EC592E06C064
:106230008FE9860D8A3148F589EA582E560C852D4E
:1062400090E08C179D070CF56F3FD9F0C216D3066E
:10625000E406F50698F0C501B4010E945A2F9B018F
:10626000AC01852D90E0A0E0B0E0280F391F4A1F57
:106270005B1F281739074A075B0710F46FEF01C04F
:1062800061E03196D1016C90C5CF0115110551F037
:10629000662311F0319703C071FE04C03297D80114
:1062A000ED93FC9370FE07C0509540953095219575
:1062B0003F4F4F4F5F4F67FF10C082E290E09093D7
:1062C0009106809390066FEF7FEF8FEF9FEF07C0EF
:1062D00060E070E080E090E002C0B901CA01DF91A7
:1062E000CF911F910F91FF90EF90DF90CF90BF90D3
:1062F000AF909F908F907F906F905F903F902F9086
:106300000895FC0188279927E89421912032E9F328
:10631000293010F02E30C8F32B3241F02D3239F4F1
:10632000689404C00E94D331820F911D21912053A3
:106330002A30C0F31EF4909581959F4F08959111D6
:1063400050C0803219F089508550D0F7089548EC3C
:1063500053E00E94AC310895FA01A191B0810097F9
:1063600019F41097E1F0CD01DC01CD010D90002072
:1063700011F4C00113C0FB012191222319F0201553
:10638000D9F7F3CFFB012191201519F41E92119634
:1063900006C02223C1F70D900020A1F7D001FA0119
:1063A000A193B08308957AE0979F902D879F802DC9
:1063B000910D11240895F999FECF92BD81BDF89AEF
:1063C000992780B50895262FF999FECF1FBA92BD5F
:1063D00081BD20BD0FB6F894FA9AF99A0FBE0196C6
:0C63E0000895992788270895F894FFCFAE
:1063EC0000009206200001000000FF0002000200E5
:1063FC000200020002000200020002000200020081
:10640C0002000200020002000200028025000005CA
:10641C00400AA1204EA50020244EA52C2330C012EA
:10642C0000001A400AA1204EA5001B1E27522C2347
:10643C00308025000005400AA1204EA50020244EE6
:10644C00A52C2330004B000006400AD0009D4900CB
:10645C007B289D492C233000E1000005400A4501B2
:10646C00D7DC03B81E0EBF00232E48E801008A407B
:10647C000A6001555502AD1E20000023C801545876
:10648C002074696D656F75742100596573004E6FCA
:10649C00002C00386368004E2F41002C205B005DFF
:1064AC002028002900486F70206368616E6E656C4F
:1064BC00200020402000456E746572696E67206173
:1064CC0064617074697665206368616E6E656C20BA
:1064DC0073656C656374696F6E2C207069636B698E
:1064EC006E673A007363616E6E6572206D6F6465E2
:1064FC00004E4F5420454E41424C45440053656E6E
:10650C0064696E672073657474696E677320746F49
:10651C002052580A00526573657474696E67207353
:10652C00657474696E6773206F6E2052580A00414F
:10653C00626F727465642065646974730A00696EB5
:10654C0076616C69642073656C656374696F6E0049
:10655C000D0A496E76616C696420696E70757420E1
:10656C002D2064697363617264656421070053654F
:10657C007474696E677320736176656420746F2020
:10658C00454550524F4D0A005265766572746564EC
:10659C002073657474696E67732066726F6D204525
:1065AC004550524F4D0A004C6F6164656420666122
:1065BC0063746F72792064656661756C74730A001C
:1065CC004B657920616E64206368616E6E656C73D7
:1065DC002072616E646F6D697A65640A004F706534
:1065EC006E4C52536E6720545820737461727469E8
:1065FC006E672000206F6E20485720006D6F647509
:10660C006C65206C6F636B65643F00342B34003811
:10661C0000382B340031320031322B34003136004B
:10662C0050504D0052535349005344410053434C76
:10663C0000525844005458440041494E004C4245C5
:10664C0045500053504B54524D0053425553005338
:10665C00554D44004C4C494E440000070B0C101196
:10666C001500B7012B032F033103350338033D030A
:10667C00B7014003440349034D0351035503590328
:10668C005D0363036A036F0374038D028D028D0235
:10669C008D02160A1322312900000000FA2CFF2A61
:0866AC00A02CCD2CB22CEF2C28
:107E00000F92CDB7DEB7112484B714BE81FFF1D035
:107E100082E08093C00088E18093C10086E0809377
:107E2000C20080E18093C4008EE0CDD088249924E4
:107E3000CC24C394F5E0DF2EE1E1EE2E73E0F72EC3
:107E4000B6D0082F813479F4B2D08983C2D0898129
:107E5000823811F481E005C0813811F485E001C059
:107E600083E09ED09AC0823411F484E103C085344B
:107E700019F485E0B6D091C0853561F498D0082F0B
:107E800010E095D090E0982E8824802A912A880CC2
:107E9000991C82C0863521F484E0A3D080E0E1CF34
:107EA000843609F04CC083D082D0A82E80D0B82E62
:107EB00000E011E07CD0F80181938F01AE16D1F77C
:107EC00088D0FB2DF53489F4E0E0F1E00BC0F9999E
:107ED000FECF92BC81BC0894811C911C819180BD15
:107EE000FA9AF99AEA1598F358C08B2D863409F05E
:107EF00054C0F401F7BEE89507B600FCFDCFF401CD
:107F0000A0E0B1E02C9130E011968C91119790E0B7
:107F1000982F8827822B932B12960C01C7BEE895C9
:107F20001124329681E0A038B80761F7F401D7BE7A
:107F3000E89507B600FCFDCFE7BEE8952EC0843774
:107F4000F1F435D034D0182F32D0B82E42D0FB2DDA
:107F5000F63421F4F40105914F010CC0FB2DF534EA
:107F600049F4F999FECF92BC81BC0894811C911C04
:107F7000F89A00B5802F14D0115049F70EC08537FC
:107F800039F427D08EE10CD085E90AD08FE069CF93
:107F9000813511F488E017D01CD080E101D050CF9A
:107FA0009091C00095FFFCCF8093C600089580910A
:107FB000C00087FFFCCF8091C00084FD01C0A89560
:107FC0008091C6000895E0E6F0E098E19083808318
:107FD0000895EDDF803219F088E0F5DFFFCF84E10E
:107FE000DFCF1F93182FE3DF1150E9F7F2DF1F9166
:0E7FF0000895282E80E0E7DFEE27FF27099492
:027FFE0001057B
:0400000300007E007B
:00000001FF
